:020000040800F2
:10000000782E00207920000839800008652000083B
:1000100000000000000000000000000000000000E0
:100020000000000000000000000000005521000852
:100030000000000000000000E5200008254800083E
:10004000A5220008A5220008A5220008A522000874
:10005000A5220008A5220008A5220008A522000864
:10006000A5220008A5220008A5220008A522000854
:10007000A5220008A5220008A5220008A522000844
:10008000A5220008A5220008A5220008A522000834
:10009000A5220008A5220008A5220008A522000824
:1000A000A5220008A5220008A5220008A522000814
:0C00B000A5220008A5220008A5220008D7
:1000BC0002B4714649084900095649008E4402BCF5
:1000CC007047C04602B4714649084900095C4900B2
:1000DC008E4402BC7047C046002934D00123002254
:1000EC0010B488422CD301242407A14204D28142AB
:1000FC0002D209011B01F8E7E400A14204D28142BB
:10010C0002D249005B00F8E7884201D3401A1A4337
:10011C004C08A04202D3001B5C0822438C08A0426E
:10012C0002D3001B9C082243CC08A04202D3001B24
:10013C00DC082243002803D01B0901D00909E3E79E
:10014C00100010BC704701B5002000F00BF802BD88
:10015C000029F8D003B5FFF7C1FF0EBC4243891A42
:10016C001847C0467047C0461C2101231B04984207
:10017C0001D3000C10391B0A984201D3000A08392C
:10018C001B09984201D30009043902A2105C4018E3
:10019C007047C04604030202010101010000000087
:1001AC0000000000414208401C2101231B0498421E
:1001BC0001D3000C10391B0A984201D3000A0839EC
:1001CC001B09984201D30009043902A2105C401AA1
:1001DC007047C0461B1C1D1D1E1E1E1E1F1F1F1FF1
:1001EC001F1F1F1F002B11D1002A0FD1002900D176
:1001FC00002802D00021C943080007B4024802A11C
:10020C004018029003BDC0465DFFFFFF03B4684673
:10021C0001B5029800F039F8019B9E4602B00CBC67
:10022C007047C046D0400B00D1409C46203AD3408A
:10023C001843524263469340184370479140030061
:10024C0090409C46203A9340194352426346D34017
:10025C001943704710B5002903D1FFF785FF2030F3
:10026C0002E00800FFF780FF10BDC04603000A78CB
:10027C0001311A700133002AF9D170470023C25C96
:10028C000133002AFBD1581E7047F0B506000F0051
:10029C0015001C0085B08B4263D801D1824260D816
:1002AC0021002800FFF7D6FF390000903000FFF73F
:1002BC00D1FF009B21001B1A1A0028000393FFF7A3
:1002CC00BDFF00900191B94245D801D1B04242D84E
:1002DC00009B019C01200021039AF61AA741FFF70D
:1002EC00ADFF04000D00039B002B2BD0019B009A4B
:1002FC00DB0750081843019B5908039B9C46B942E5
:10030C002CD801D1B04229D832003B00121A8B41B3
:10031C00012692185B410027B6185F4101235B420E
:10032C009C446346002BEAD130003900039AFFF756
:10033C0079FF039AA4197D4106000F00FFF77EFF99
:10034C00241A8D410A9B002B01D01E605F60200097
:10035C00290005B0F0BD00240025C4E7B6197F4183
:10036C00DCE700240025EDE770B5294D03212800BA
:10037C00284A07F08CFD284E300008F002FB0028BC
:10038C0008D1012128001324244A07F080FD64427F
:10039C00200070BD10203169B3680A6882430A607E
:1003AC00A022042130001B6812039847041E06DAB1
:1003BC001B4A23000121280007F070FDE8E700F03C
:1003CC002BF9041E01DA174AF3E700F0EDFA041ECC
:1003DC0001D0154AEDE700F031F8041E01DA134A9A
:1003EC00E7E700F025FA041E01DA114AE1E70321E0
:1003FC002800104A07F04BFDB36810215B693000F0
:10040C00984700F037F800210B4806F053FBF3E750
:10041C00209200088A950008888F0008B89500087B
:10042C00D4950008F59500081B9600083F96000827
:10043C0064960008889600088813000010B50948D7
:10044C0008F09FFA031E084806D10121074A07F05D
:10045C001EFD1320404210BD0321054A07F017FD75
:10046C000020F8E7C88F0008E8910008AE96000855
:10047C00C7960008F0B5A7B0444B03939B681B6864
:10048C00002B07D00F2502AAAD1829000398984716
:10049C00041E01D027B0F0BD3D4F2A783B680A2AD4
:1004AC0001D00D2A68D1002BE6DD0022394E3A49E5
:1004BC00F2543000083208F0EFFB06AD002808D1EA
:1004CC000121080000F0EAF834492800FFF7CEFEBD
:1004DC0040E033490922300008F0DEFB011E04D154
:1004EC00012000F0DBF82F49EFE7082230002E49FD
:1004FC0008F0D2FB002805D10121023000F0CEF823
:10050C002A49E2E72A490922300008F0C5FB011EFE
:10051C0004D1022000F0C2F82649D6E706223000AA
:10052C00254908F0B9FB00281CD1013000F006F970
:10053C00224E002800D0224E022000F0FFF81F4B64
:10054C00002800D01E4B00938021330028001D4A48
:10055C0006F054FE2800FFF791FEA04204D80023B9
:10056C003B6089E71849B0E7295D039B03989B68BA
:10057C0001345B689847EDE73E2B04DC591C39606D
:10058C000449CA5478E73C6076E7C046C88F000837
:10059C00F807002030120020DF960008E8960008CB
:1005AC00F3960008FD9600080997000812970008BA
:1005BC001D9700082797000833970008F996000844
:1005CC00E59600083A970008519700080300F7B524
:1005DC0019790068DB88826894460269DC0715D4B7
:1005EC00B0246403234301273D000A4C16681C40C9
:1005FC008D4001943400AC433B4201D034002C4379
:10060C00634614601B68019A9847FEBDD0246403AE
:10061C006340E8E7FFFFEFFF70B5174808F0B1F94A
:10062C00164D002808D1012128001324144A07F084
:10063C002EFC6442200070BD124808F0A2F900287C
:10064C00F1D01148FFF7C2FF041E06DA0F4A23004F
:10065C000121280007F022FCECE70D48FFF7B6FF5C
:10066C00041E01DA0B4AF2E7032128000A4A07F0BC
:10067C000EFC0024DEE7C046A88F0008309200086C
:10068C0076970008888F00089C92000892970008C3
:10069C0094920008B4970008D6970008B0B50C00E7
:1006AC0000AF012820D11B4807F03BF8002819D1D6
:1006BC00194B1C70194B002C00D0194B6C4688B090
:1006CC006A461849936180239B009383164B5161B2
:1006DC001361E621154800231032490101F096F808
:1006EC000020A546BD46B0BD02280FD1104807F02A
:1006FC0018F80028F6D10F4B1C70084B002C00D0BA
:10070C00074B6C4688B06A460B49DBE71620404223
:10071C00E8E7C0469C92000871120020F996000888
:10072C00E5960008EF9700080300000130920008DE
:10073C009492000870120020F8970008030001281A
:10074C0002D1044B187870470020022BFBD1024BCE
:10075C00F8E7C0467112002070120020082390B5F3
:10076C0087B000AF0C00F8180021102208F08CFAAA
:10077C00012321685B423B6079606379DA0703D51A
:10078C00802212060A437A609A0704D5802279687F
:10079C00D2050A437A605A0701D50222BA721A07A7
:1007AC0003D50422B97A0A43BA72DB0603D50823AF
:1007BC00BA7A1343BB7223793B7208F005FA0A220A
:1007CC000023FFF70FFDFA239B0043437B61237942
:1007DC001A1C082B00D908220C232100F818D2B2BD
:1007EC00083108F048FA1821380000F099F86379BC
:1007FC008AB05B0720682179DB0F6A4653620623B7
:10080C00084CD0615461084C116294611361C4218D
:10081C00002306481032890100F0F8FFBD4607B0EE
:10082C0090BDC0460E980008A098000800920008E1
:10083C00F0B587B01C4F380008F0A3F81B4E002809
:10084C0009D1012130001324194A07F020FB64421E
:10085C00200007B0F0BD0A226846164908F00BFAD2
:10086C006946380007F080FC041E06DA124A2300A1
:10087C000121300007F012FBEAE70025012203AB4F
:10088C001A7238002A000D4903955D6002F088F851
:10089C000400A84201DA0A4AE9E703213000094AB8
:1008AC0007F0F5FA2C00D3E7E88F00080092000857
:1008BC002D980008889200084298000869070008E3
:1008CC005F9800087F9800080122054B10B51A703C
:1008DC0004480321044A07F0DAFA002010BDC04690
:1008EC007212002068920008BB98000880B500AF17
:1008FC0088B06A46074BC8215361074B93610323A9
:10090C001361002305481032490100F07FFFBD46FA
:10091C0080BDC046E1980008DE9900086892000886
:10092C00B0B50E4B00AF1B78002B14D06C4688B0C2
:10093C006A460B4BD16153610A4B936104231361DB
:10094C008421094800231032890100F05FFF002048
:10095C00A546BD46B0BD80204042FAE77212002089
:10096C0003990008F69900086892000870B50B4DC1
:10097C00032128000A4A07F08AFAFFF759FF041EE0
:10098C0007D001210300074A280007F087FA20004E
:10099C0070BDFFF799FF0400F9E7C04668920008A4
:1009AC002E9900085F99000810B50A4C032120000D
:1009BC00094A07F06CFA8120084907F075FB031E01
:1009CC0004D001212000064A07F068FAFFF7CEFF99
:1009DC0010BDC04668920008869900085D77000833
:1009EC00BB990008F0B597B0059304230B921A40FD
:1009FC000B9B0A92DA0807231A40013207001C9D50
:100A0C0003910D92820700D0C5E1041D002804D08B
:100A1C00072909D81C20404254E1039A1A401300BC
:100A2C00A4180822D31A0393059B0426013B0693B2
:100A3C00002309930C9304930293013B07930196B3
:100A4C00002F01D0059B23600D9B002B00DDF1E0F6
:100A5C009D4B059A9A4203D39C4B9A4200D2E9E0F3
:100A6C000B99E21B9308890700D50DE1049A0F2A14
:100A7C0000D9BBE0002F00D10EE104990EAA53540B
:100A8C000A00079912AB99540C9B01330C93F4E0B8
:100A9C0008260196069B01330693069B987800283E
:100AAC0000D105E1029B002B08D12528F2D1079B30
:100ABC0001330793012302930426EAE77A284AD8E4
:100ACC004B280ED8472846D829282CD825283FD083
:100ADC0041D82028DED0233843425841C3B2029378
:100AEC00D8E74C382E2836D8FFF7E2FAD43535350E
:100AFC003535353535353535373535353535353598
:100B0C003561353737616161D437D235D435183713
:100B1C0018353579E63735353735E6000023089337
:100B2C000426029327E0012213002A38C0B2834026
:100B3C0067490B42AED1E2211800890508400B42EF
:100B4C0035D11900114002911342A3D0089013E043
:100B5C00079B013B07930023C1E70022069B0892E9
:100B6C005B7802926C2B07D10426069B01961B78AE
:100B7C006C2B01D1B6190196013CA0193100FFF77D
:100B8C00ABFA70430400002F3BD0019B039ADB1B94
:100B9C001B18934200D93DE7089B002B41D1019BC8
:100BAC00042B20D108CD03600423043415E0072165
:100BBC0007358D4364188C430CCD002F08D00131C0
:100BCC00C91B03980919814200D923E7226063608D
:100BDC000023082602933300083401935AE7029B42
:100BEC00089300239CE7019B082B01D0162012E7E9
:100BFC00072307359D430CCD02604360082308345E
:100C0C00EBE7089B002B0CD1019B042B01D1043585
:100C1C00CAE7019B082BE9D10735013B9D430835F9
:100C2C00ECE7069B023306930D9B013B0D9308CD1D
:100C3C00059305E70B9B9B0722D50121E21B93082B
:100C4C00802080008242D1D2049A0F2ACED8002F65
:100C5C001CD00498DBB20EAA13549C46079B12AA14
:100C6C001354002900D10FE78022634652421343EC
:100C7C000EAA1354099B01330993049B013304936B
:100C8C00069B0434013B07E70021D9E7002903D078
:100C9C00039B01330393F0E7039B023303930A9BFB
:100CAC00002BEAD10598FFF7E9FA039B1B18F1E733
:100CBC008022E31BD200934298D2002F0AD10398D2
:100CCC000838C01817B0F0BD108E0008F0A6000848
:100CDC00DAFF00009B08302238603B706B469B1893
:100CEC000A9A1B78002A0BD0FB70099BBB70002B57
:100CFC001BD100250EAE049BAB421BD1E01BE1E7E0
:100D0C007B70F2E70EADED560EA9595C002D07DA9B
:100D1C00039E15190140B54200D97BE621700134C0
:100D2C00013304999942EDD1E3E7012200237F209E
:100D3C00D21BF6E7099B002B02D033787F2B1BD8F4
:100D4C000A9B002B1BD012ABEB5C237000230134ED
:100D5C0001930123019ADB1B1B199B18039A9342E5
:100D6C0000D957E63378019A237001342000059995
:100D7C0007F081FF019B1C1901350136BBE7337865
:100D8C009B00FB181A6805920A9A05981A60FFF7DF
:100D9C0075FA431CDCE70E203DE6C046F0B59BB06F
:100DAC0000AF3B628023FB181B6806001B07DB0FA0
:100DBC007B618378F9623A63BB6300290AD10478BA
:100DCC00BB6BA400E41845780419FB6A9D421BD840
:100DDC00A31BFB62F378BB61BB6B002B04D080239D
:100DEC00FB181B68DB0719D4BB69002B47D13B6B85
:100DFC00002B03D030003A6AF96A9847FB6AFB6310
:100E0C00BD46F86B1BB0F0BD01342000FFF736FA7D
:100E1C00FB6A013001332418FB62D6E73378FB619F
:100E2C009B007B627368BB627B6AF5183B6B002B83
:100E3C0000D029E1FB6AFB63BB6BEC180023BB639E
:100E4C00A54232D02B789B009859FFF717FA8421D2
:100E5C007B181B680130002B0CD08822BA18BB6B96
:100E6C001268934206D27A1812685B009852BB6BD8
:100E7C000133BB63FB6B01351B18FB63E0E780237D
:100E8C00FB181B689B07B2D53378FB619B007B6218
:100E9C007368BB627B6AF5183B6B002B77D1FB6ADE
:100EAC00FB63BB6BEC183B6BBB6380220523BA184E
:100EBC001268250013405A4253410133FB62BB694F
:100ECC005B00E3183B633B6BAB4299D02B787B63A5
:100EDC006B789B009C59B84B9C4202D3B74B9C42FD
:100EEC0023D37B69002B33D0796BB86A06F0D0FC26
:100EFC0000282DD06C468AB06A46B14B5361BB6A50
:100F0C0093617B6BD36180239B001384AD4B136186
:100F1C0092210023AC481032890100F077FCA546E1
:100F2C00FB6B023BFB630235CDE77B69002B05D0E5
:100F3C00796BB86A06F0ACFC0028DBD18023012267
:100F4C00FB181B68134209D1FB6BFA6A9B1AE9E781
:100F5C0080230222FB181B681342E4D02000FFF709
:100F6C008DF984217B181B68002B0DD08822BA18B0
:100F7C00BB6B1268934207D2791809685B00421C5C
:100F8C005A52BB6B0133BB63FB6B1B18CAE7BB6BC1
:100F9C001C1E7B6315D0802104237A1812681A401A
:100FAC0014007A637A1812681A420AD00023BC6BB8
:100FBC007B63183340229B182900BA6BD81907F0B1
:100FCC005AFEBB6BEB18FB60FB63BB695B003B61C0
:100FDC003A69FB68944663447B60FB6B7A68934286
:100FEC0057D17B6B757800215A198023FB181B682D
:100FFC00D2B29B0700D46108802038180068002307
:10100C00C00705D48033FB181B685B07DB17234034
:10101C007270B370F17030003A6A796A3B6B984722
:10102C00F863002800DAEBE6FB6940203370BB6BF9
:10103C002100B370BB693A6AF37018231B18D819D6
:10104C0075703B6B9847041E00DAB1E0FB6ABA6B13
:10105C00F868991A7B6A3A6AC91A3B699C46C91A9C
:10106C0060443B6B9847002800DAA3E00025FB6B3B
:10107C001C192318FB637B6B9D4261D300213A6AD8
:10108C0008003B6B9847BBE6BB6B00247B630823D3
:10109C0090E7FB6B484A1B78BB60FB6B5D78AB0041
:1010AC009B59934202D3454A93420CD37B69002B44
:1010BC0030D0B968B86A06F0EBFB00282AD0FB6B7D
:1010CC000233FB6389E77B69002B05D0B968B86AEA
:1010DC0006F0DEFB0028F2D180230122FB181B68EE
:1010EC0013420AD07B6B9B18073240215218796B44
:1010FC00D219DBB255547B63E1E78023FB181B68E4
:10110C005B07DCD5182240215218631CD2191555E7
:10111C00DCB2D4E780230222FB181B68134203D0F5
:10112C007B6B06320133E0E7402118225218B96874
:10113C00631CD2191155DBB20234E4B2D554BEE7AC
:10114C00402208239B18DB19EB5C0732BA1813708A
:10115C0084229B009B59BB63BB181C68002C09D0D4
:10116C008823FB181B6800249D4203D2BA1812680E
:10117C006B00D45A47230121F8183A6A3B6B984705
:10118C00002817DBFB6B1B18FB63002C04D1B86B1E
:10119C00FFF774F8013084B221003A6AB86B3B6BEC
:1011AC009847002806DBFB6B01351B18FB6362E7D5
:1011BC00F86325E6F86323E6108E0008F0A6000815
:1011CC001B9A000804000001E0910008014B186014
:1011DC007047C04600000020F7B504000D001E004B
:1011EC00019205F0A7FC030007F002FE054F320048
:1011FC003B5001992800A04707F0FAFD385800F041
:10120C004FFFC04608000000802102200A4B090550
:10121C00DA6B82B00A43DA63DA6B0A40074901924F
:10122C00019A4A68824300204A60DA6B04490A40FA
:10123C00DA6302B07047C04600100240005801400B
:10124C00FFFFFFF780230D4A9B00116882B00B4310
:10125C00012113600A4B0B4A1A600B4B1A6C0A43A0
:10126C001A641B6C094A0B400193019BC023116843
:10127C00DB000B43136002B07047C04600200240F5
:10128C00300000200024F400001002400000014057
:10129C00F7B505000600002D01D13000FEBD280079
:1012AC00FEF780FF01238340DA430E4F04019D4378
:1012BC003B1901931B7B0092002BECD0E3591B696B
:1012CC00002B09D1009B3C191E406368042219684D
:1012DC00019806F09FFDDEE7381998470028DAD10F
:1012EC00F0E7C04678920008F0B5002289B00F49AB
:1012FC000F4807F06DFC0024002600270E20C022AA
:10130C000C4D03900696079728000B4B0B49049441
:10131C00029401940094920005F032F908492800D7
:10132C0007F078FB200009B0F0BDC046511300084F
:10133C00B005002038010020551600087812002056
:10134C00E39A000810B5024804F08EFF10BDC046A9
:10135C00B8000020F7B500901F48019106F039FD48
:10136C00061E35D000252800FEBD237B002B11D096
:10137C002368DB68002B01D02000984763689F71BD
:10138C0023681B69002B1BD1636804222000196899
:10139C0006F040FD01361034104B9C42E5D3009B07
:1013AC00002BE0D0002DDDD02800FFF771FF019B52
:1013BC000500002BF6D00021642005F07BFBF1E743
:1013CC00200098470028DFD03B00B3401D43E1E7E5
:1013DC0005000127024CDFE70C080020889200086A
:1013EC0078920008014B8000C0587047B8920008F2
:1013FC00030010B50800002B05D0044A136000F060
:10140C00ABFC002010BD16204042FBE7040000207E
:10141C0010B5054C2378002B02D1044804F024FFAE
:10142C000123237010BDC04673120020B8000020A9
:10143C0010B50400074806F0CCFC002C03D00121A9
:10144C00054807F0F7FB054807F0CEFB044804F00D
:10145C000BFF10BD0408002008080020B005002078
:10146C00B800002010B50021014807F0F0FB10BDBA
:10147C000408002070B5FFF7F5FF0500084C094B78
:10148C009C4200D370BD63685B79002B06D0236847
:10149C005B68002B02D02900200098471034EEE73F
:1014AC00789200088892000810B5044C044920007A
:1014BC0006F01FFB034B1C6010BDC04668000020EB
:1014CC00A4920008FC0700200023FA210C4A10B556
:1014DC0013700C4A890013600B4A0C481360FFF719
:1014EC0087FFFFF7E1FF0A4B0A4918008B4200D334
:1014FC0010BD1A1A5C681211013222711033F5E713
:10150C00741200200408002008080020E97D00085F
:10151C00789200088892000810B5044C0100002253
:10152C000023200006F006FB10BDC046680000201A
:10153C0010B5024806F098FB10BDC04668000020AC
:10154C0010B5034B0100186806F0DFFB10BDC04658
:10155C00FC07002010B5024806F010FC10BDC04678
:10156C006800002070B5204B1878002826D0FFF7B3
:10157C00DFFF1E4C051E2CD11D4B1E4C1B68002B77
:10158C0011DD07F021FB0A220023FEF72BFE226857
:10159C006368801A9941002903D1FA239B00984271
:1015AC0001D9FFF767FF22686368FA2000218000E9
:1015BC0012184B4122606360FFF7CCFF70BD63686B
:1015CC005B79002B04D02368290020001B68984706
:1015DC001034094B9C42F2D32800FFF7B1FF0121D4
:1015EC00064807F027FBC7E7731200207892000823
:1015FC0004080020A8050020889200080808002094
:10160C0070B50E4D297800290CD10120FFF7A2FEF0
:10161C000B4C0C4B9C4206D3FFF7A4FF0028FBD1CC
:10162C0001232B7070BD63685B79002B03D023689A
:10163C0020009B6898471034EBE7C04674120020DA
:10164C007892000888920008F7B500210800FFF78F
:10165C0081FE041E2DD0FA2700267F0007F0C8FB60
:10166C001C4B1D4A1B581360002B06D01B4B1B68D0
:10167C00092B02DD1A4804F0F7FD00230093002C1F
:10168C0007D02000FFF704FE041E02D101277F4281
:10169C003E00FFF767FF0190002808D1009B114D19
:1016AC00002B13D10E483A00330004F00FFE019BBF
:1016BC00E4E701277F423E00D0E72B689B69002BB3
:1016CC0003D000222800110098471035064B9D428C
:1016DC00F3D3E7E70800000000080020080800200A
:1016EC00B8000020789200088892000813B51548BD
:1016FC0006F06FFB144B1B78002B0AD0EFF3108411
:10170C0072B6FFF72FFF002C02D162B6BFF36F8FBA
:10171C0013BD0E4B1B68002BFAD0002809D10022F8
:10172C0000230B480092019300230A4A05F012FD96
:10173C00EEE70928ECD1064807F056FA064804F003
:10174C0093FDE5E708080020741200200008002033
:10175C00B005002010270000B800002010B5064B83
:10176C0004001B6898472100A060044806F060FA4A
:10177C00FFF7BCFF10BDC04604000020680000202D
:10178C00044B054A00209B1ADB08994201D2C90080
:10179C008858704778920008C8910008F0B55E1C14
:1017AC0085B0B5000090280007231730984303300C
:1017BC0080080F000192FFF7AFFE02AB040003227A
:1017CC00581D002107F060FA03AB1E70002C0BD0E3
:1017DC00039B21002361002314312A1F0198C05858
:1017EC00C85004339A42F9D1E023BA015B001A4085
:1017FC006D02054B2A431A4020000023009906F085
:10180C002DFB05B0F0BDC046C0FF0F00F0B591B088
:10181C0004AF3B600B035B0D0D0078607A613B619C
:10182C000C0D002B00D173E0BB60002604237E62FC
:10183C00BE62FE6202931833FB1801930A2318222E
:10184C00009302339B18DB193200B9687869FFF7F3
:10185C00A5FA8023F8601B01984224D37B696C465F
:10186C001A795B798AB01B0213437A699279120454
:10187C001A437B69DB791B06134304AA9361294B3A
:10188C002949D36180239B001384284B5161136138
:10189C0092213300264810328901FFF7B7FFA54685
:1018AC00BD460DB0F0BDFB6817345B055A0D3A61AF
:1018BC00204A1B0B15401D43FB68E0180723984377
:1018CC0003308008FFF728FE041E15D003001033E8
:1018DC007B62FB68FE62BB62042302931833FB1825
:1018EC0001930A231821009302335B18124AB9683A
:1018FC007869DB19FFF752FA3B690E4A5B02154017
:10190C001D432A0020003B68796806F0A7FAC7E758
:10191C00200007231730984303308008FFF7FCFDA5
:10192C000400E9E7FF070000F89A00080400000132
:10193C0008920008FF01F0FF377E0008F0B587B071
:10194C000E9F0400150002910393002F15D00F9BDE
:10195C0010210593009300203B000D9AFFF742F8ED
:10196C00802306001B01984208D30221174A18480D
:10197C00184B06F093FA07B0F0BD3E000723220087
:10198C000C9C1D401A40D2001734AD011543A01910
:10199C007202154398430C9A0330120580081543C4
:1019AC00FFF7BAFD041E09D0002F07D00F9B3100A2
:1019BC0000930D9A3B001030FFF714F82A0020001A
:1019CC00039B029906F04AFAD5E7C046379B0008FC
:1019DC0008920008FF0700004068002804D0044B60
:1019EC00C01AC00800B2704701204042FBE7C04655
:1019FC00C89100080EB417B5054C05AB04CB01001B
:101A0C002000019300F058FC1EBC08BC03B0184722
:101A1C00057F000810B5CB0604D4890603D503490D
:101A2C00FFF7E8FF10BD0249FAE7C0460797000828
:101A3C0006970008F0B591B0079317AB1B7804001C
:101A4C000D0006920593002B00D1B4E002261B9BDF
:101A5C001B9A1E4001231A400C921B9A07331A4002
:101A6C0008921B9AF8331A400992002706F0D0F915
:101A7C000200B84204D020008D49FFF7BBFF0700DD
:101A8C00002E09D044231B9A1A4235D12A0020007B
:101A9C008849FFF7AFFF3F180C9B002B0AD0059A23
:101AAC00854B9200D258002A00D1844A20008449E8
:101ABC00FFF7A0FF099B002B5AD0089B002B77D176
:101ACC001D00069B002B05D01A0020007D49FFF756
:101ADC0091FF0500189B7C48ED19002B00D0BEE04F
:101AEC001A9B002B74D11B9BDB0700D5DAE020007E
:101AFC001B99FFF78FFFBEE00020744B1E688642D7
:101B0C00C9D0734B28001968FEF7E6FAFA253100A4
:101B1C00FEF71EFBAD0069430A9008003100FEF78A
:101B2C0017FB0E91E1210D9009010A98FEF710FBAD
:101B3C000B910B983C21FEF7CFFAE1210F90090194
:101B4C000A98FEF7C9FA0A900E9831006843FEF71E
:101B5C00C3FA0D9B02903C210B980193FEF7F8FA07
:101B6C00200000910F9B0A9A5A49FFF743FF92E716
:101B7C00089B099D002B08D0059A574B920020001A
:101B8C005649D258FFF736FF0500069B002B05D0AF
:101B9C001A0020004B49FFF72DFF2D18079B002B37
:101BAC0098D01A0020004E49FFF724FF2D1891E71A
:101BBC0000230793E0E7079B4A48012B00D14248DA
:101BCC00189B059D002B4AD11A9B002B53D0002546
:101BDC001A9F102F00D9102720001B99FFF71AFF0E
:101BEC000026B5424CDC199B20001A783E49FFF7C1
:101BFC0001FF012607231E4203D120003B49FFF7BA
:101C0C00F9FEB74242D9199B20009A5D3649FFF77D
:101C1C00F1FE0136102EEDD1002620003449FFF7DD
:101C2C00E9FE3300199AD25C1300203B5E2B00D9DD
:101C3C002E2220002F49FFF7DDFE0136102E2AD070
:101C4C0007231E4203D120002849FFF7D3FE33009F
:101C5C00B742E7D820002549FFF7CCFEEDE7189BEB
:101C6C002200254905F0E0FD1A9B002BB0D1059B05
:101C7C00002B00D037E7200006F032F911B0F0BD90
:101C8C0020001A49FFF7B6FE0136AAE720001B49CF
:101C9C00FFF7B0FEBDE7199BDB1919931A9BDB1BF1
:101CAC001A93E2E72000054A0549FFF7A3FE1EE759
:101CBC00749B0008789B0008C89200086F9B000872
:101CCC00F59700089D9B0008057F0008140800206C
:101CDC0010080020819B0008DC920008A19B0008E2
:101CEC00A79B00082B7F0008AC9B0008B49B000846
:101CFC00B69B0008B89B0008C5220008B29B0008E0
:101D0C0073B5114A04000B000568914200D9130009
:101D1C00052168460D4A05F071FA06006368280033
:101D2C000B220B495B6806F0CCF863683200280084
:101D3C0069465B6806F0C5F8636828001B220549F4
:101D4C005B6806F0BEF873BD0F270000329E0008DA
:101D5C00D79B0008BB9B0008012310B500211C0079
:101D6C00074A904207D8074A002900D10123136083
:101D7C00054B186010BD210040085B00F1E7C04620
:101D8C0040420F00100800201408002070B50D0010
:101D9C0004004618B44201D1280070BD21780348D4
:101DAC00013483685B689847F4E7C046C88F000825
:101DBC0010B5034A03480021121A06F029F910BD88
:101DCC0078120020380100200648074A10B5121A74
:101DDC00064906F021F9064A06480749121A06F088
:101DEC001BF910BD0000002037010020F0A60008F0
:101DFC000000002000000020F0A60008F0B585B01F
:101E0C0000AF0C1EB86036D06E468AB06D460968BD
:101E1C006268A3682B6205232048A9616861EA61A6
:101E2C002B61A1212A001E481032002389017A60FF
:101E3C00F860FFF7EBFCB546E168AD4622696369D3
:101E4C002B6205231748A9616861EA612B61A12106
:101E5C0000237A68F8688901FFF7D8FCB546E36976
:101E6C000121114AF86806F019F8A36901210F4AFB
:101E7C00F86806F013F8BB68012B07D1EFF3058364
:101E8C000B4A0748B968103B06F008F82100B868FF
:101E9C0003F0B0FFBD4605B0F0BDC046449C000841
:101EAC0028920008739C0008A29C0008B19C0008B2
:101EBC00DF9C000830BFFDE7F7B50A4B0A4D060062
:101ECC00EF18CC1B2A0020000849019306F0D3FE22
:101EDC0060190021019A06F0D7FE3800083C7466A0
:101EEC000830FEBD040000000000000088920008CD
:101EFC00054B5A699B689A4205D08023034A5B05BF
:101F0C0051680B4353607047FC11002000ED00E05A
:101F1C00F0B53E4B8BB05B6800AF7B60DB05DB0D37
:101F2C0004003B6062B6BFF36F8F394E130EFF2B6C
:101F3C0008D1F33B1340082B3DD101213000354A29
:101F4C0005F0A5FF00252C003B68032B39D1324A44
:101F5C000121300005F09BFFA369304A934202D364
:101F6C002F4A934205D32F4A934249D32E4A934288
:101F7C0046D2023B1A882D4B9A4241D1236801214B
:101F8C0030002B4A05F08AFF266808232022F81817
:101F9C00210006F070FE7B6A002D33D0DA0502D1E9
:101FAC00244A13437B6208233000F918FFF726FFFD
:101FBC00BD460BB0F0BD01251207C5D50C000025A0
:101FCC00C2E7F822796852001B4B114200D01B4B20
:101FDC006A468AB07A606A4693613B681849103B3E
:101FEC00D36180239B001384164B516113619121A3
:101FFC000023300010328901FFF708FC7B689D46F6
:10200C000026C2E75B0A5B02CCE7C04600ED00E0AD
:10201C0028920008209D00084B9D0008BC00000879
:10202C00088E0008000000200000002002DF0000E5
:10203C00629D0008FF010000F29C0008079D00084B
:10204C007E9D0008040000010821024A53698B435D
:10205C005361704700ED00E0EFF30880EFF3098166
:10206C0001B57246FFF754FF01BDC046094880F325
:10207C00088872B608480949401880F30988EFF3BC
:10208C0014800221084380F31488BFF36F8F05F08E
:10209C00D9FF0000782E00207815002000080000E1
:1020AC0010B50A4B9B6883420DD1EFF30583002BCF
:1020BC0009D08022064B520559680A435A605A6A65
:1020CC0004490A405A6204F03BFD10BDFC1100208B
:1020DC0000ED00E0FF7FFFFF15498A6815481044AA
:1020EC00EFF3098CF0C043464C4655465E466746B6
:1020FC00F8C072B6104F114E4A698A603E60104C9F
:10210C00141920680F4C2060906E002393660028F1
:10211C0000D162B6074C10191030F8C89846A14689
:10212C00AA46B346BC462438F0C88CF309887047DD
:10213C00FC1100203000000004ED00E0000000085D
:10214C00640000003C08002004207146014202D0CB
:10215C00EFF3098001D1EFF3088081690239097826
:10216C000229FFD001B5724605F05AFF01BDC046E9
:10217C0043B2000605D41F221A4001239340014AA2
:10218C001360704700E100E030B5FF2503220B001F
:10219C00290040B20240D20091409B012B40C94320
:1021AC00934000280ADBC0240A4A8008800080186B
:1021BC00A40002590A401343035130BD0F221040B2
:1021CC000838054A800880008018C26911401943FC
:1021DC00C161F2E700E100E000ED00E0FF22044BFA
:1021EC009343044A9360BFF34F8FBFF36F8F7047D5
:1021FC000000000800ED00E010B5203A1360029BCF
:10220C0001245360039B06499360049BA143D36054
:10221C0080235B04D361002391610265836610BD4A
:10222C00E511000870B50B4B15009860426E0A4B17
:10223C000E001A602C1C86F309880020034B98476B
:10224C00201C002100220023014C20476D80000837
:10225C00E5110008FC1100203C0800201022014B65
:10226C001A61704700ED00E0F0B5C024002203268F
:10227C00FF25A40010002F003040C0008740054906
:10228C0093089B005B1819590132B94319511F2A45
:10229C00F0D1F0BD00E100E010B5EFF30583054A85
:1022AC00103BDB00D118496898588847FFF720FE8F
:1022BC0010BDC04608900008F0B587B007000E00AE
:1022CC0014000021102268461D0006F0DDFC6A4651
:1022DC0002239370054B2A00210068460193049752
:1022EC00059604F0B5FF07B0F0BDC0468780000826
:1022FC0010B5024B1B689847002010BD4008002009
:10230C00034B044A1860022391780B439370704777
:10231C004008002010000020072310B50449054A8E
:10232C0099430548521A05F045FA002010BDC046E5
:10233C007F5200200040022044080020F8B506001F
:10234C00002501277378AB4200D8F8BD34786419A6
:10235C00200000F0FDF800280ED0200000F022F93B
:10236C00074AE1008B58002B06D052181F21380069
:10237C000C40A040516898470135EDB2E2E7C046E9
:10238C00500800200022052010B50C4C11002070C4
:10239C006070FFF7F9FE002206201100A070E070BB
:1023AC00FFF7F2FE0C220721054806F06DFC002217
:1023BC0007201100FFF7E8FE002010BD40000020B0
:1023CC004400002010B50400FF20002C05D0200094
:1023DC00FDF7CAFE1F23181AC0B2044B1856044B43
:1023EC00DA6F1443DC67FFF7C3FE10BD400000201A
:1023FC0004180240024AD36F8343D3677047C04628
:10240C0004180240020000B5080003290AD80E4B3C
:10241C00FDF758FE02090C131968914319605968AD
:10242C009143596000BD19681143F7E7596811438E
:10243C005960196891431960F4E7196811431960E0
:10244C0059680A435A60EDE70018024070B5FF2343
:10245C000D001400002804D0FDF786FE1F231B1A64
:10246C00DBB2094AD8008358AB4203D11118496832
:10247C00A14204D0002B04D1155012185460002036
:10248C0070BD10204042FBE750080020FF2310B520
:10249C00002804D0FDF768FE1F231B1ADBB20021B5
:1024AC00024ADB009950D218516010BD5008002030
:1024BC00C022C30452031340032210B50724800822
:1024CC0003431A401B0C9C4099400448920012187C
:1024DC00106EA0430843106610BDC04600180240A1
:1024EC00C022C304520313400322800803431A4042
:1024FC00044918329200505807221B0C9A40104085
:10250C00D84070470018024013B50E4C200006F05E
:10251C0038FA002807D10C4801210C4A05F0B7FC09
:10252C00132040420AE0402300933F3B0193A368F1
:10253C001B68002B03D069462000984716BD582015
:10254C00EFE7C046A88E0008F09100089E9D000899
:10255C001F220121024003000800904010B5020028
:10256C003F2B05D90C480D4A05F098FC002010BDF6
:10257C000B481F2B0AD8C36813409A4204D0016938
:10258C001140891A4B4259410800F0E7C36A1340C5
:10259C009A42F9D0016BF3E7F0910008BD9D000859
:1025AC00001802401F22012102400300080010B550
:1025BC0090403F2B06D90848084A05F06FFC1620BE
:1025CC00404210BD064A1F2B03D8D060106100207A
:1025DC00F7E7D0621063FAE7F0910008BD9D0008A0
:1025EC00001802400200802103008A430020072AC1
:1025FC0008DC5AB20448002A00DA044824228B432F
:10260C005343C0187047C046B40B0020D40C0020B4
:10261C0010B5024802F04EFA10BDC046D00800209A
:10262C00044B020010B51800034905F036FD1620C6
:10263C00404210BD50920008FD9D0008130042B2AC
:10264C0013B50400002A0BDA802801D1002B0AD024
:10265C0011482200114905F020FD1620404216BDFC
:10266C00402B00D940238022210091430C4A0D4875
:10267C00890189180A18210006F03EF90300002090
:10268C008342ECD00448009301212300064A05F054
:10269C000DFC0520E2E7C04650920008FD9D0008A5
:1026AC0024050000D00800200F9E000843B210B58E
:1026BC000C00002B01DB002902D1FFF7B1FF10BD8C
:1026CC00034B0100180006F032F920600020F6E7F9
:1026DC00D008002070B5114C00234022802120002E
:1026EC0006F0DEF80023402219002000902606F0A8
:1026FC00D7F8002576008323DB00E0184019243539
:10270C0003F0B2FDB542F6D1B8239B00E358002B81
:10271C0002D000210120984770BDC046D00800208F
:10272C00B82210B5044B92009B58002B02D000210C
:10273C000520984710BDC046D0080020B82210B51F
:10274C00044B92009B58002B02D000210620984786
:10275C0010BDC046D0080020BC23082270B5104C18
:10276C000025104E9B00E25032000433E5500E4B16
:10277C0003CB03C2BB239B00E358AB420ED0290012
:10278C0028009847094BE25AAA4207D0063BE35C63
:10279C007F2B03D831002800FFF750FF70BDC046D7
:1027AC00D0080020F40D00206C0B0020A2020000C9
:1027BC00F0B591B0029316AB069204CB03911B8833
:1027CC0004920193029B5C889B880134E418029B61
:1027DC00DB88E418002A00D1D4E0FA23019A9B008C
:1027EC009A4200D3CEE083680FA99B6A98470028D1
:1027FC0000D0C9E0019B002B0CD1644B049A9A4287
:10280C0040D8634B93429B414A229343614A94467E
:10281C00634401930F9B0499180061430D93FDF7DA
:10282C005BFC069B1B89984200D21800049B059008
:10283C0043430C93584B0A93029B059A1B89934272
:10284C0022DA0A98039B039ADB8892885B08191C8E
:10285C00934200D9111C039B8AB21980069B1B88DA
:10286C009A4206D9029B19880B1C914200D9131C61
:10287C009BB2039A1380484B984201D18620404268
:10288C0011B0F0BD454BC4E70C990D98FDF760FCF9
:10289C000990002930D1029BFA219B88890007936B
:1028AC00029B5B880B930B9A079B9C18069BA4B20C
:1028BC009B880893069B5D886B469E8C019B5843B6
:1028CC00FDF70AFC069B301ADA8880B2170090429A
:1028DC0006D9029BDB881F1C834200D9071CBFB2A0
:1028EC00731EDB1B9BB29C420FD2029B361B013E1C
:1028FC00DB88B7B2BB4212D2049A059B94460133D3
:10290C0005930C9B63440C9396E708994C19A4B25D
:10291C009C4217D9361B013EB7B2BA42ECD86308B9
:10292C009D4206D26A46958D0B9A9A4200D91D1C7F
:10293C00ADB2661B079BB6B2B34205D2E51A1E00B8
:10294C00ADB204E01C00EAE7089BB342F6D8FA23C8
:10295C00601C9B0058430999FDF7BEFB019A0300CC
:10296C00101A9A4200D2981A0A9B9842C4D2039B1E
:10297C00059A5D809E80DF801A81002800D161E776
:10298C000A90B9E716207AE7052078E700350C00A5
:10299C0020A107006B030000FFFFFF7FEE02000089
:1029AC00F7B5846800AFA446002928D0002B26D0A8
:1029BC001C7A1E685D68E40725D58024A405A64210
:1029CC0001D2A54229D31D21082316486A468EB090
:1029DC007A606A461362936280239B00124C1386C2
:1029EC00124B54619061D1615662D5621361002320
:1029FC000F4810491032FEF709FF7B689D461620E0
:102A0C004042BD46FEBD80242401A64201D2A5420F
:102A1C0003D30B2103230848D8E76446A469A047D5
:102A2C00EFE7C046429E0008819E000808000001A6
:102A3C00C8910008404400004B9E000873B5140078
:102A4C001D0082683032064E83683A33B44204D893
:102A5C0001950094FFF7ACFE76BD16204042FBE7D3
:102A6C0040420F0073B514001D0082684832064EB8
:102A7C0083685233B44204D801950094FFF798FE52
:102A8C0076BD16204042FBE700127A0037B543684A
:102A9C000D009B691B689847041E06D001212B0072
:102AAC00034A0448009405F001FA20003EBDC046DC
:102ABC00CE9E0008D091000837B543680D009B6985
:102ACC005B689847041E06D001212B00034A04487A
:102ADC00009405F0EBF920003EBDC046F19E0008C5
:102AEC00D0910008F0B59BB00393436805000291A8
:102AFC0001920021482208A8DF6906F0C5F82800D9
:102B0C00019905AAFFF7C2FF002818D17F22059B67
:102B1C00134214D03F2248241B0A1A405443029BF0
:102B2C0000921C19A4B206AA08232100280005F063
:102B3C0044FB021E05D03C493C4805F054FB1BB03D
:102B4C00F0BD04AB9B7B1B071B0FDAB2944608AAA3
:102B5C00137104ABDB7A990603D50221507901433A
:102B6C00517106AA9279910604D5042108A84679D8
:102B7C0031434171D20604D5082208A94879024391
:102B8C004A715AB2002A04DA102208A94879024381
:102B9C004A7106A9CE7908AA7606760E5B061FD571
:102BAC00069BDB00DB080893012351790B4353711F
:102BBC0062461F4B9B5C402B2FD808AA5279920778
:102BCC0013D4002B11D00322033308349343280071
:102BDC000AAAA1B205F0F1FA021E06D01549ABE71C
:102BEC004B88DB045B0D0893E2E708A94B79F600F0
:102BFC00DB0710D5BB689E1933687268002B01D0B7
:102C0C00280098472800009A0399FFF755FF0028E1
:102C1C0000D174E793E77B68EDE70121064A03488E
:102C2C0005F0DDFAEEE7C046159F0008D0910008CC
:102C3C009AA300083C9F0008619F0008F7B50500A7
:102C4C00066901225242D3171036300005F0D2FA31
:102C5C001821280001AAFFF719FF041E28D1102300
:102C6C00019A18219A4328000192FFF725FF041EB0
:102C7C001ED101F0A1FE1821070001AA2800FFF7C0
:102C8C0005FF041E14D10822019B134210D001F041
:102C9C0093FE0E4BC01B98420FD91022019B18219A
:102CAC001A4328000192FFF707FF041E00D10B3CCA
:102CBC00300005F0A3FA2000FEBD1821280001AA5F
:102CCC00FFF7E4FE0028DED00400F1E700A8610065
:102CDC0070B50469050023790E00002B25D1103442
:102CEC0001225242D317200005F084FA7F21F38889
:102CFC003288013B0B40FF21013A52061A43B3883C
:102D0C000902013B1B020B401A4333890849013B62
:102D1C001B040B4028001C211A43FFF7CDFE0500B5
:102D2C00200005F06BFA280070BD10256D42FAE703
:102D3C000000FF01F0B5036987B001931B79050012
:102D4C004768002B00D06AE0386800280ED08368F2
:102D5C00019A1B6811689847041E07D0220031495C
:102D6C00314805F040FA200007B0F0BD2E69012271
:102D7C005242D3171036300005F03CFA18212800C7
:102D8C0005AAFFF783FE041E0ED0300005F036FABC
:102D9C0025482200254905F026FA38680028E2D09B
:102DAC0083685B689847DEE70123059A18219A43EC
:102DBC0028000592FFF780FE041EE6D105F004FF03
:102DCC00029003912800182105AAFFF75FFE041E4C
:102DDC00DBD10122059B134208D1300005F00EFA1D
:102DEC00002CD5D10123019A1371BCE705F0ECFE40
:102DFC00029A039B801A994100290DDC03D1FA2316
:102E0C009B00984208D81821280005AAFFF73EFE1F
:102E1C000028DED00400E0E70B246442DDE77824D0
:102E2C006442A0E7729F0008D09100089C9F0008A4
:102E3C00F0B506000D00076985B0072907D92A00EF
:102E4C002A492B4805F0CFF98624644242E03B79AD
:102E5C00002B48D13B0010330193019801225242C0
:102E6C00D31705F0C7F91821300002AAFFF70EFEA0
:102E7C00041E2CD11021300003AAFFF707FE041EFC
:102E8C0025D18022029BE90727D51A4310230292F1
:102E9C00039A13430393029B20211A008A43A80729
:102EAC0001D50A001A436B071AD5C0239B001A439D
:102EBC00182130000292FFF7FFFD041E07D11021EC
:102ECC003000039AFFF7F8FD041E00D13D60019815
:102EDC0005F094F9200005B0F0BD93430293DAE7B6
:102EEC00044B1A40E4E71024AFE7C046BF9F00082C
:102EFC00D0910008FFFCFFFFF7B5502101AA040098
:102F0C004768FFF7C3FD002835D199260125019BA1
:102F1C001A00324033422ED050212000FFF7CCFD56
:102F2C00002828D1019B2B4205D0A823A4222000E5
:102F3C00F98EFFF7D7FD019BDB0605D5B823B4222C
:102F4C002000398FFFF7CEFD019B1B0704D529000C
:102F5C00094A0A4805F043F9019B1B0604D52900D0
:102F6C00074A064805F03BF95021200001AAFFF75B
:102F7C008DFD0028CBD0F7BDD89F0008D09100085C
:102F8C00EE9F0008F0B5040003698BB0029350214A
:102F9C00200006AAFFF77AFD002805D106995F4BA1
:102FAC000A001A40194201D10BB0F0BD502120008B
:102FBC00FFF782FD0028F7D1E022069B9204134212
:102FCC0037D026692000B36807AA0093F3680393EF
:102FDC006368DF6904ABDD1D290005F0B5F9002835
:102FEC0027D12B780193009B002B05D02000039B4D
:102FFC00079A0199009DA847019B032B19D1012227
:10300C00D42120005242FFF757FD051E11D13B7B06
:10301C009D4254D31821200008AAFFF737FD002841
:10302C0007D10123089A18219A4320000892FFF730
:10303C0043FD8022069B5201134222D06768FB6934
:10304C00009323690193F421200007AAFFF71EFDCA
:10305C00002816D13F23079D1D4212D01F232D0A95
:10306C00B98F1D40EB00C91808AE320008232000B0
:10307C0089B205F0A2F8021E36D02949294805F07C
:10308C00B2F8069B1B0408D50121274A254805F0F8
:10309C00A6F80298243003F0E7F8069B9B0004D5B1
:1030AC000121224A1F4805F09AF8069B9B0300D485
:1030BC006DE701211E4A1B4805F091F867E73A6855
:1030CC00E90052181368002B0CD0002010603A68ED
:1030DC00200052187221526849429847300024301F
:1030EC0003F0C2F8013592E72A00F8212000F679A6
:1030FC00FFF7E2FC051EC4D1009BF6001B689B1970
:10310C005A681E68039218600198243003F0ACF8DA
:10311C0029002000039AB04795E7C0460090823BF7
:10312C0004A00008D09100082AA000083FA00008C5
:10313C005AA00008F0B58FB0099343680792069324
:10314C00039004910C79DF690669784A231C0F2CD3
:10315C0000D90F23DBB2D35C002108220CA8059305
:10316C0005F092FD01214025049BAC465A79530889
:10317C000B40900128405B01034308A8C3748023D3
:10318C00D008313D084025405B4200012B430343EE
:10319C0090080840400103436046834308A88375A8
:1031AC000F2A06D96249634805F01DF8862464424B
:1031BC00B3E033685B0707D40C231A4204D05E4A91
:1031CC005C4805F00CF8F1E7059B402B09D940232E
:1031DC0001210093594A5748059B04F067FE1624B9
:1031EC00E5E7520707D50F2C08D95549220051485D
:1031FC0004F0F9FFF3E75349082CF7D83379002B87
:10320C0000D18DE0442103980BAAFFF73FFC041E6C
:10321C0000D082E00B9B1B0600D583E033002433E7
:10322C000893079A099B089803F050F8041E00D0E5
:10323C007AE0343601225242D3173000079604F05C
:10324C00D9FF3B7BA34241DC0126764204990CAAB0
:10325C00D671049B49791B68C9073FD50C9ADB00D2
:10326C00520FDB08520713430C9348257543069BFA
:10327C00ADB2D98F0398691889B208230CAA04F04F
:10328C00A2FF3149041E16D1049B5B799B072DD4F8
:10329C00059B002B2AD0032206990333C98F934335
:1032AC000831049A69180398083289B204F08BFF2C
:1032BC00041E1BD0254922001E4804F094FF0798D9
:1032CC0004F09CFF089802F0CFFF26E03A68E1007A
:1032DC008A582600002AB9D00134B3E751881C481B
:1032EC005B05DB0C01400B435380BEE73B68149A33
:1032FC00F5005A513B68159A5B195A600122D0218E
:10330C00B2400398FFF7D8FB041E03D000223B68A1
:10331C005A51D4E7079804F071FF20000FB0F0BDAC
:10332C00732444E7722442E70B2440E79AA3000875
:10333C0075A00008D091000898A00008C3A0000850
:10334C00F3A0000815A1000837A1000861A100082E
:10335C0003E0FFFFF0B587B0039242680291D76992
:10336C0001921A682A4912040A40802100245B68E1
:10337C0006695B0509065B0D0B431A431036059273
:10338C00050001225242D3173000009604F032FFA0
:10339C007B7BA3420ADC1C2502211E4A1E4804F03A
:1033AC001EFF009804F02AFF6D422DE07A68E600BB
:1033BC00B258002A0DD00134EBE7009804F01EFF40
:1033CC007B68029A25009A517B68039A9B195A6074
:1033DC001AE00123382004AAD17923400133814318
:1033EC00DB000B43D371019AA300518E2800C9183E
:1033FC0089B2042305AA04F0E6FE051EDDD02A00DE
:10340C000649054804F0EFFE280007B0F0BDC046A1
:10341C000000FF07B5A10008D091000889A10008A1
:10342C00F0B51D00436887B00291039201932A7A8C
:10343C000400DE69012A06D93A493B4804F0D3FE60
:10344C00862464426AE0002A43D004AB0769052253
:10345C000021D81C05F018FC2A68049BD2005B0FD5
:10346C00D2085B0713430493802380216A680025EC
:10347C00D200D2081B061343059A89050A40134350
:10348C0010370593380001225242D317009704F0ED
:10349C00B1FEB37B9D4209DB0221244A224804F091
:1034AC009EFE009804F0AAFE1C24CAE7B268EF0046
:1034BC00BA58002A14D00135ECE7009804F09EFEAF
:1034CC00B368029A2C00DA51B368039ADB195A607C
:1034DC0022E02B00039A0299FFF73CFF04001DE049
:1034EC0001231F2104AAD2782B4001330A405B012F
:1034FC00134304AAD370019B2000998E0823C91989
:10350C0089B204F060FE041ED7D022000849064898
:10351C0004F069FE002C01DB737BE418200007B07B
:10352C00F0BDC046D5A10008D0910008F9A1000853
:10353C0089A10008F7B5436805000C1EDE69076910
:10354C00019305DA22002049204804F04CFEF7BD17
:10355C00103701225242D317380004F04BFE727B15
:10356C0094421ADBB37B1849A21A934228DD00213E
:10357C00B368D2009950B36828009B185960019B1E
:10358C00998E891889B2082204F023FE1049021E74
:10359C0016D1380004F032FED9E700227368E1003E
:1035AC005A507368A4005B185A60019B0432598E00
:1035BC002800091989B204F00CFE021EE9D0054955
:1035CC00024804F010FEE4E719A20008D0910008AC
:1035DC0034A2000860A20008F8B504694568237994
:1035EC000600EF69002B46D0FA220023920004F06B
:1035FC0009FE002807D00121204A214804F0EFFDE4
:10360C0005256D420CE0286800280BD083685B68A8
:10361C009847051E06D02A001A49194804F0E3FD04
:10362C002800F8BD0025300004F0CFFE25713B7B4F
:10363C009D420BD3103401225242D317200004F0C8
:10364C00D9FD200004F0DAFD0025E9E73A68E9002D
:10365C0052181368002B0CD0002010603A68300010
:10366C00521873215268494298472000243002F0C6
:10367C00FBFD0135DBE77825C3E7C0468CA20008CB
:10368C00D0910008A6A20008F0B589B0456806697B
:10369C0004000A22002102A8EF6905F0F5FA0A22BB
:1036AC00002105A805F0F0FA3000103005F08CF977
:1036BC003000343005F088F9397B30000A002430B2
:1036CC0005F089F9286800280AD005F05AF9002875
:1036DC0006D101214F4A504804F081FD132013E01C
:1036EC002000FFF7ABFA4D4A002808D1FA2200233C
:1036FC002000920004F086FD002808D0484A464875
:10370C00012104F06CFD0520404209B0F0BD200001
:10371C0004F05BFE1821200001AAFFF7B7F900287E
:10372C00F3D1019A3F4B18211A4020000192FFF768
:10373C00C3F90028E9D11021200001AAFFF7A6F94E
:10374C000028E2D11021019A20008A430192FFF750
:10375C00B3F90028D9D18021200001AAFFF796F9EE
:10376C000028D2D12B22019B80211A4320000192E8
:10377C00FFF7A2F90028C8D1EA682B8A200002A919
:10378C00FFF75CF9284A1630B9D06A696B8A2000B9
:10379C0005A9FFF767F9254A1630B0D0200002A919
:1037AC0004F0E2FC021E04D021491B4804F01BFD6E
:1037BC0094E705A9200004F0E9FC1E49021EF4D18F
:1037CC001D4A542120000192FFF776F900289CD164
:1037DC009922582120000192FFF76EF9002800D0A1
:1037EC0093E703225C2120000192FFF765F9002882
:1037FC0000D08AE70122E021524220000192FFF71B
:10380C005BF9002800D080E701002A6C200004F04E
:10381C00E0FC7AE7EBA20008D0910008D1A20008E6
:10382C008CA200085BFCFFFF05A3000827A300087F
:10383C0053A3000871A3000899908203D02843D0A9
:10384C002BD8A82842D011D884281CD00300883B40
:10385C009BB21C2B20D801229A4026490A4212D135
:10386C00082B35D01C2B17D1902015E0B82831D05F
:10387C000BD8B42830D00FD803000422AC3B9343B0
:10388C009BB2002B08D11C4806E0CC2826D003D8CC
:10389C00BC28F8D0C828F6D07047E02820D007D82C
:1038AC00D8281FD0DC281FD0D428F5D1D020F3E79E
:1038BC00F4281BD004D8E4281AD0F028E3D0EBE786
:1038CC00F828E9D1E820E7E7CC20E5E79420E3E706
:1038DC008420E1E79C20DFE79820DDE7C820DBE7C8
:1038EC00DC20D9E7D420D7E7D820D5E7E420D3E7EC
:1038FC00E020D1E701001101FFFF000070B5436823
:10390C0008005E6C0D001400FFF798FF1D4B9842E9
:10391C0034D03368C0180368582D1FD019D804222E
:10392C009543502D17D1FF22F82099019205114093
:10393C00C002DA00024011430122FE201A4011435A
:10394C0040019A00024011431C225B0013400B43C0
:10395C0001E0802D0FD02360002070BD02211A00E1
:10396C000A400B4200D0D022DB0701D42260F3E7DF
:10397C000D231343EFE73F221340ECE78620404230
:10398C00EBE7C046FFFF000070B5436808005D6CB4
:10399C000E001400FFF752FF1C4B984232D0582EE9
:1039AC0021D019D804239E43502E17D1FF22F82181
:1039BC00A309120413400902E2080A40134301222E
:1039CC00FE2122401343C900A2080A4013430E22D1
:1039DC00640814401C4301E0802E0FD02B68C018E3
:1039EC000460002070BDD02323405A1E93410D2249
:1039FC0022405C000123002AECD1EFE73F23234057
:103A0C00034CE7E786204042ECE7C046FFFF00008E
:103A1C0000001C08F0B5436885B05B6C0500002104
:103A2C00586903AA009304F06EFE041E07DB039B87
:103A3C0000221979186800F035FB041E08DA344AA4
:103A4C0023000121334804F029FA200005B0F0BD11
:103A5C006B685E6C304F380004F093FF002851D037
:103A6C00BB68F1680193B368012B13D9019B083132
:103A7C009B69002B0BD0002238009847041E09DAF2
:103A8C000121264A234804F002FA254AD8E7582493
:103A9C006442F5E7019BF1681B68002B35D03800B8
:103AAC009847041EF1DB337E002B06D0280004F06F
:103ABC008CFC337E1B4A5B081360280004F085FCE9
:103ACC008021280003AAFEF7E1FF041EBDD1039B51
:103ADC00154A80211A4328000392FEF7EDFF041EBD
:103AEC00B3D18022C02128005204FEF7E5FF041E4A
:103AFC00ABD12800FFF7C8FD041EA6D1009B1B69A3
:103B0C009847A2E713246442BFE75824FBE7C0465A
:103B1C00B3A30008D8910008A88E0008D1A3000810
:103B2C00FBA300080065004000001C0873B5436847
:103B3C000C005E6C1A4D280004F023FF00282CD0DA
:103B4C00AB68B268F168DB68012A17D90831002B21
:103B5C0007D1144A1448012104F099F90520404278
:103B6C000BE0280001AA98470028F2DB0F4B0198C4
:103B7C001A68002A0CD12060002076BD002B01D1E0
:103B8C000B4AE7E7280001AA98470028EEDAF7E786
:103B9C0019684900FCF7A0FAEDE71320DFE7C046EF
:103BAC00A88E00081CA40008D891000800650040ED
:103BBC0048A40008024B18684005C00F7047C04667
:103BCC00001002400B8813B50C481B051A0D1B186E
:103BDC001B0D0C2B0ED80A4C486813191A6802439B
:103BEC0000201A600B881B051B0D1B191B68019309
:103BFC00019B16BD86204042FBE7C0460000C0FC7E
:103C0C00001002400B8809481B051A0D1B181B0DD0
:103C1C000C2B07D80020064B4968D3181A688A4326
:103C2C001A60704786204042FBE7C0460000C0FC8B
:103C3C000010024070B508881F4B00050D001400E1
:103C4C001B68000D0C2818D8002801D1863870BDCF
:103C5C0002380A2809D8FCF735FA2606222426262B
:103C6C0008081D1D1D00FA23DB0180222360296832
:103C7C005201914219D20020E9E7104A8018000540
:103C8C00000D0C2803D80E4AC240D207EDD4862072
:103C9C004042DCE700F02AF9C3005B08E5E7094B7A
:103CAC00E3E7094BE1E70023DFE7090B18000131DB
:103CBC00FCF712FA2060DEE730000020CC0F000089
:103CCC00111100000024F400006CDC020C2806D852
:103CDC00044BC3400020DB0700D486387047862095
:103CEC004042FBE73A1F000070B508880C00000545
:103CFC00000DFFF7EBFF00281EDB6368FF2B1AD0CB
:103D0C0001225802800F013082401F2099B21B0CF7
:103D1C000340013A9A40094E89190D6895430D608C
:103D2C00636899B21A0E1B0C03409A401300891950
:103D3C000C6823430B60002070BDC046001002408D
:103D4C000B880A4A1B05180D9B1810B51B0D0C2B64
:103D5C0008D8074BC0180368486898434342584139
:103D6C00013010BDFFF7B2FFF8E7C0460000C0FC01
:103D7C0000100240F7B5524F00F0D0F8380004F0B4
:103D8C0080FB00F02BFE1F214E4C4F4AA3683D00D8
:103D9C001B051B0F9B009B580B40D84013680190D0
:103DAC000B401D41A84202D2280001F0EBFFFFF7A7
:103DBC0001FF012808D0802322685B001343236095
:103DCC00FFF7F8FE0128FBD12368404A134023601B
:103DDC000123226E134323660223226E1A42FCD067
:103DEC0080232268DB031343236080231B04226897
:103DFC001A42FCD03822A3681340102B18D1FFF7BD
:103E0C00D9FE012808D0802322685B00134323606D
:103E1C00FFF7D0FE0128FBD10722A3689343A360D0
:103E2C003823A2681A42FCD1A368294A1340A36024
:103E3C002368284A1340802223609204236813428B
:103E4C00FCD1254B25491868802608408021890221
:103E5C0001431960802118684902014319601968EF
:103E6C001F48760401400A431A601A6832431A60EC
:103E7C0000F040F823681E43802326609B042268D0
:103E8C001A42FCD0A368124A1340A3600723A2680D
:103E9C009A43053B13433822A360A3681340102BAD
:103EAC00FBD1019BAB4202D3280001F06BFF0D4B01
:103EBC000D4A1F60A36800201340A360FEBDC046DE
:103ECC000090D003001002400C950008FFC7FFFFC4
:103EDC00FFF0FFFFFFFFFFFE0C100240FFFFC1FFD2
:103EEC00FFFFFFF130000020FF8FFFFF00487047FD
:103EFC000024F400064B074AD9681140064A0A43CD
:103F0C00DA608022D96852050A43DA607047C046ED
:103F1C00001002408C80FF1F0208002080210F4BF4
:103F2C004905DA6B82B00A43DA63DA6B0A40802106
:103F3C000192019ADA6B49020A43DA634022DB6B85
:103F4C000B400093009B064B19680A431A60202211
:103F5C0019680A431A6002B07047C046001002404C
:103F6C00006C004010B5084804F00BFD002808D088
:103F7C00064C2000FEF7C4F92000FDF727F90020BD
:103F8C0010BD13204042FBE7C88F00089D3F00087E
:103F9C0070B50400074D0A2804D1AB680D21280028
:103FAC005B689847AB6828005B68E1B298472000D3
:103FBC0070BDC046C88F0008F7B547681E0003697E
:103FCC00B868009201930C0004F062F88023009A08
:103FDC0005009B039A4215D12000BD68FEF780FABC
:103FEC0085420DD12100280004F052F80400FEF7A0
:103FFC0001FA2000FEF74AFA00212000FEF702FA2F
:10400C000020FEBD8023009ADB039A4224D080233B
:10401C00DB049E421CD0C023DB049E421AD08023BA
:10402C0016209B049E4218D1022628000D49019AA5
:10403C00FEF70CFA002812D12000B968FEF738FA06
:10404C0028003100FEF7DEF92800FEF7BBF9D7E7B0
:10405C000126EAE70326E8E786204042D1E7102054
:10406C00FBE7C046B786000870B5036904005860CA
:10407C000B4D280004F085FC00280FD0AB6861685C
:10408C001B680C31002B04D028009847002803DC57
:10409C0070BD58204042FBE70020F9E71320F9E7F8
:1040AC00A88E0008F7B504000025C9004318019339
:1040BC00019B9C4201D1002035E01F271023226870
:1040CC0017401A4217D1202563681D43F821530964
:1040DC0049000B40E2395209FF390A401A43009259
:1040EC001B09192B20D8114A9B009E58002E0AD16F
:1040FC001320404217E0102F03D0112FE6D1656832
:10410C00E4E73025E2E7300004F03BFC0028EFD078
:10411C000F2300992A00194030003B0004F0DEFA0E
:10412C0008340028C4DAFEBD1620E2E754940008D7
:10413C0070B50369C0225B680C001B68D2000B6071
:10414C008021436805001B68C9001B6813400222CC
:10415C008B4204D01C4A9B185A425341DAB2C021FC
:10416C00802022716B6889011B6800225B6840010A
:10417C000B40834206D002328B4203D0013A002B13
:10418C0000D0023262716B681B6818681968C02312
:10419C00DB0019400D4B184004F0FFFAC022A0714F
:1041AC006B6892001B689B681340094A9B185A4223
:1041BC005341DBB2E3716A6812689268520400D50D
:1041CC0003230020E37170BD00FAFFFF0010001004
:1041DC0000FDFFFFF0B5436885B000AF05001E6819
:1041EC0002697960002939D01068D9688368DB6866
:1041FC00002B0DD00C22BA189847041E0BDA0121A3
:10420C001A4A1B4803F043FE2000BD4605B0F0BD22
:10421C0058246442F3E73368164A796813403360D4
:10422C007B685808FB68C018FBF756FF0F2818D896
:10423C006C468AB02B686A4693617B680E49D361E1
:10424C0080239B0013840D4B51611361912100233A
:10425C00074810328901FDF7D9FAA54616246442A5
:10426C00D2E780B20024F060CEE7C046FFA400087D
:10427C0048920008FF7FFFFF2DA5000804000001F5
:10428C00F7B50C00036941685D682379012B13D0E5
:10429C009A1E56427241920200926679022E0ED8F4
:1042AC00494F7600F75BA679022E0BD0042E34D042
:1042BC005E1EB3411B0308E0C022D200ECE780274E
:1042CC00BF01F0E75E4273411B07E67901960026B9
:1042DC00B446019E012E02D1C026B600B446096830
:1042EC00A5421DD10C68394E009A34402243134329
:1042FC000B604B68364A13403B434B60436835496F
:10430C001A6893680B4061460B4393602968FFF76A
:10431C0061FF002800DD0020FEBD80235B01D4E797
:10432C00C0220E68D2001640009AB24205D00E6828
:10433C00294A1640009A16430E60C0264268B60100
:10434C0011684A683240974204D04A68204E324085
:10435C003A434A604268214E11680A6832409342DF
:10436C0004D00A681E4E324013430B60C0214368D0
:10437C0089001A6893680B409C4505D093681549D1
:10438C000B4061460B43936080224368D2011B684B
:10439C009968114206D0019A032A09D09A681149EA
:1043AC000A4004E00199032902D199680A439A60F2
:1043BC0021682B689942AED0FFF70CFF0028ABDBCD
:1043CC0023682B60A7E7C04684950008FFE9FFEF40
:1043DC00FFCFFFFFFFFCFFFFFFF9FFFF00100010F6
:1043EC00FFEFFFEFFFBFFFFFF0B506004568046964
:1043FC00744885B000AF206004F0C3FA002806D1E1
:10440C00714A0121714803F042FD13240BE020682E
:10441C00E96883681B68002B07D101216C4A6B4843
:10442C0003F035FD582464420AE09847041E0BD172
:10443C000C230021286AFA1804F065F9041E0BDA23
:10444C002000BD4605B0F0BD0121614A5F4803F074
:10445C001EFD002CF4DBEBE7FB68002219791868D1
:10446C00FFF720FE041EEBDB0122756833692C6814
:10447C005B687B60236893432360686804F081FA6F
:10448C00002801D1534ABCE76868A9688368DB68D7
:10449C00002B00D09847EFF31082012383F3108890
:1044AC000C2123680B43236082F310883000796859
:1044BC00FFF7E6FE002801DA1624B4E72B7D002B6B
:1044CC0003D00823A2681343A3606B7D002B04D098
:1044DC0080226368120213436360AB7D002B04D00F
:1044EC0080226368520213436360EB7D002B04D07F
:1044FC00802263689202134363602B7E002B49D0A9
:10450C00354B9C4229D0354B9C4226D0344B9C4297
:10451C0023D0344B9C4220D0334B9C421DD0334B88
:10452C009C421AD0324B9C4217D0324B9C4214D036
:10453C006C4688B06A463368936180239B002E4991
:10454C0093832E4B51611361E22100231F481032DB
:10455C004901FDF75BF9A546AEE773681A6880233D
:10456C009168DB010B43936022686B7E24495B05E9
:10457C000A40134323602268AB7E22491B040A4085
:10458C0013432360EB7E002B04D08022A36812021D
:10459C001343A3602B7F002B04D0802322689B0540
:1045AC0013432360012322681343236080239B035E
:1045BC00E2691A42FCD08023DB03E2691A42FCD088
:1045CC0000243DE7A88E000844A500084892000886
:1045DC0063A5000883A50008003801400044004092
:1045EC0000480040004C004000500040003C01409E
:1045FC0000800040008400409EA5000803000001DC
:10460C00FFFF1FFCFFFFE0FFF7B5436800901C683D
:10461C0003690D005B6801934B790A799C46887994
:10462C00012A16D1022B2ED9C02180230600C900E5
:10463C009B01022800D188E0042836D00020824259
:10464C0037D08020033A4001012A32D886204042DC
:10465C00FEBD022A09D1022B23D980210600C900F4
:10466C00022860D080239B01E6E7022B1BD90600B1
:10467C0000210228F6D10021002A54D180201100FB
:10468C00400503221AE0C021C9006646344B76006F
:10469C00F35A06000228CFD1002A56D180204005BB
:1046AC0007E08021F0E70021EFE7002ACED180203F
:1046BC004001802700227F01BB423CD16245C5D11D
:1046CC0004F06BF8B042C1D1EB79002B19D0012B5F
:1046DC0042D1244B9C4214D0234B9C4211D0234BEF
:1046EC009C420ED0224B9C420BD0224B9C4208D0B9
:1046FC00214B9C4205D0214B9C4202D0204B9C422A
:10470C00A4D1012623682900B34300982360FFF746
:10471C00B7FD00289ADB236800201E43019B26600E
:10472C0006CD06C394E7033A012A00D88EE780230E
:10473C00002002269B01C0270222BF01BB42BDD034
:10474C00013A002BBAD00232B8E7033A012A00D85A
:10475C007CE702260020ACE7032BBAD076E7C046F4
:10476C008495000800380140004400400048004097
:10477C00004C004000500040003C014000800040D4
:10478C000084004070B580251049114B8C681B6863
:10479C000E6810488A686D02002C08D1002A11D1CD
:1047AC001A002E4209D100681818801A70BD002A10
:1047BC000AD02E4201D1A242F5D90468E418046053
:1047CC000968F0E71C00F4E71A00F2E710E000E0DB
:1047DC00F8110020F41100200A4A0020136A1B0271
:1047EC001B0A1362C822084B52011A60074B084A75
:1047FC001860084B5A600722986019680A431A60BF
:10480C007047C04600ED00E0F8110020F4110020C4
:10481C00FF18000010E000E0F8B50024FFF7B2FF2D
:10482C00104E23003168104D0A0028686968801802
:10483C00594128606960C8210C4D346049012E68CB
:10484C006F68801BFBF748FCC821490141432300DA
:10485C000A0092197B412A606B6002F077FBFDF72E
:10486C0047FBF8BDF4110020F0050020E8050020FE
:10487C00F0B53B4B3B4D87B0002960D0421C08D1B2
:10488C0001212A688A432A60FF2212061A6007B0A7
:10489C00F0BD1B68039300230293012854DCEFF353
:1048AC001083059372B6FFF76DFF00221100AB6801
:1048BC0004932D4B1E685F6836184F413000390049
:1048CC0018605960294B009601971A60284B1C6898
:1048DC00009B1B1B93423EDBC82702987F01784349
:1048EC00244A39008018C018FBF7F6FB009B78436C
:1048FC00E41A80232018DB00984200D218001E4BCB
:10490C00984200D91800164B174918600138AB684B
:10491C0068600020A860049AD41A9A421ED2039DA3
:10492C00621903000C684D6812196B410A604B60E8
:10493C00059B002BABD162B6BFF36F8FA7E71B684B
:10494C000393431CA7D10D480D4B984200DD180072
:10495C00431E0293A3E78020C000D4E72200E0E7C7
:10496C00F811002010E000E0F0050020F411002008
:10497C00E8050020FF18000000DCFF003C0A0000E6
:10498C003D0A000070B5EFF3108572B6084A094B6A
:10499C0014681B68E41AFFF7F5FE0019002D02D10C
:1049AC0062B6BFF36F8FC8214901FBF795FB70BD51
:1049BC00F0050020E805002070B5EFF3108572B605
:1049CC00054B1C68FFF7DEFE2018002D02D162B6E5
:1049DC00BFF36F8F70BDC046F0050020382370B553
:1049EC001D4CA2681A4205D123681C489B045B0F1E
:1049FC00D84070BDA2681A40082A27D0A2681A4075
:104A0C00102A17D1E368E168DB43E5684906490FD2
:104A1C006F322D0A013115409B0709D11048FBF765
:104A2C005BFBE1686843490F0131FBF755FBE0E79D
:104A3C000A48F4E7A2681A40202A09D0A26800208C
:104A4C001340182BD5D1FA20C001D2E70448D0E787
:104A5C0080200002CDE7C046001002400024F40084
:104A6C0000127A000A2382B00193019B002B07D11C
:104A7C00054BC000C01800688001800D02B0704763
:104A8C00019B013BF0E7C046009800400A2382B02E
:104A9C000193019B002B07D1054BC000C018406847
:104AAC008001800D02B07047019B013BF0E7C046CE
:104ABC0000980040F0B5040087B0006803F046FF92
:104ACC00CA4B1A6804231A420ED0802580222D026C
:104ADC0012020540104201D100F032FC8022256800
:104AEC0012026B6C134201D107B0F0BD0F270F22DD
:104AFC006B6C1F40134200D0A4E01900013211402E
:104B0C00134221D12B68BA4A200013408022120292
:104B1C0013432B60237DB74ADB009B181B68A26AEA
:104B2C009B019B0D2363D318A36203F0DEFA637C15
:104B3C00002BD3D0E26A2168002ACFD18020637C7D
:104B4C000343CB646274C9E72B6880221E001201F8
:104B5C00164013421BD0AA235B00E05CFFF796FFC4
:104B6C002200A7215532FF3289000300D061611861
:104B7C002800D28801F0D8F821689F4B0A682000E1
:104B8C001A40802313430B60FDF7E6FDA6E71B04D8
:104B9C00A4D52A68984B1A40802313432B60AA2370
:104BAC0025005B00E05C2768FFF770FF5535FF358B
:104BBC00031EE8610ED0696900290BD03800EA8821
:104BCC0001F0B2F86B69EA6931009B1820006B6147
:104BDC0003F076FA23681B681A0500D57EE7C0221D
:104BEC0092011340934200D178E7824A53689B01AB
:104BFC009B0953602B693E2B17D91F205909034081
:104C0C0058424341C91A53688906194380231B062D
:104C1C000B4353602168794A0B681340C022920100
:104C2C005A40774B13430B6058E7002B01D1516866
:104C3C00ECE7012059080340C91853688906194349
:104C4C005160E7E7BB00ED1801932B6803936B46AB
:104C5C009B890293039B1B043ED52A68664B1A4022
:104C6C00802313432B6028257D4365192B0061336A
:104C7C00FF331A78236804932B005533FF33002A33
:104C8C0069D11878FFF702FF0190002809D02B009A
:104C9C005B33FF33FC351A88E96E0300049801F08E
:104CAC0043F82823190079436218FC32506F019D98
:104CBC0040195067D06E4019D066106F002803D091
:104CCC00926E954200D3FDE07B43E3185533FF33DE
:104CDC002000197803F0F4F9039B22681B0600D41A
:104CEC00FCE6BB00D218136841490B408021090235
:104CFC000B4313602823190079436618F27D012AAF
:104D0C0000D018E17A1C53430022E3185A60731C3C
:104D1C00DB7F934217D0039B5B0600D4E8E0737DE6
:104D2C00934200D0D5E0337D3249DB005B181A6822
:104D3C00920192091A608022337D1206DB005B1807
:104D4C0019680A431A6028237B43E318197D200055
:104D5C0003F0CBF9C2E62A005832FF3212781E78E3
:104D6C00022A00D086E08023029ADB011A400592C9
:104D7C00029A3000FC351A4248D0FFF773FE2A6FB6
:104D8C0003000190824222D3121A2A6721D0029A80
:104D9C0052060ED528227A43A2185532FF321178CA
:104DAC0022688900521810681649084016490143B8
:104DBC001160002B00D174E72821794361180A0097
:104DCC005D32FF32FC311288C96E206867E7002221
:104DDC002A67049AB6009619326808490A4080215D
:104DEC0089015140064A0A433260D0E7A0000140D5
:104DFC000F8FFF07009800408F0FFF078FBFFF0733
:104E0C00808000008F8FFF07C0800000FFF73EFE00
:104E1C002A6F0300019082421DD3121A2A671CD0FC
:104E2C00029A52060ED428227A43A2185532FF3227
:104E3C0011782268890052181068C6490840C64982
:104E4C0001431160002B00D12BE728217943611815
:104E5C000A005F32B5E7059A2A67049AB6009619DC
:104E6C003268BE490A40802189015140BC4A0A433C
:104E7C003260D5E7049AB60096193168B54A1140EC
:104E8C00B54A0A433260187826688300F3181B6809
:104E9C005B040ED5FFF7E6FD0190002800D100E77A
:104EAC002B005D33FF33FC351A88E96E03003000AC
:104EBC00F5E6FFF7EBFD0190002800D1F1E62B00A1
:104ECC005F33EFE75531FF312068611800F068FC63
:104EDC0002E7012B00D036E7337DA249DB005B18DB
:104EEC001A6892B21A60337DDB005B181A6829E7E6
:104EFC00737D002B10D1337D9A49DB005B185A6807
:104F0C00920192095A608022337D1206DB005B18F5
:104F1C0059680A435A6016E7012B00D013E7337D1A
:104F2C009049DB005B185A6892B25A60337DDB0003
:104F3C005B185A68EEE780230398039A5B00357D73
:104F4C0018401A4219D1874AEB009B181B68F26A69
:104F5C009B019B0D9A4202D82900F062F7E6D21A07
:104F6C00F262B26A1431D218B262326B6118D31881
:104F7C003363206800F014FCB0E52368029A0393B5
:104F8C0040231A400192029A28001A4200D1EDE007
:104F9C00FFF768FD8022F36AD201834214D8002304
:104FAC00F362029B13400193737D002B52D0012BB3
:104FBC005FD16C4AED00AD182B689BB22B60337D32
:104FCC00DB009B181A6853E01B1AF362029B134216
:104FDC0000D087E028227A43A218150038352B78A8
:104FEC00012B00D006E1936A1B189362336B1B18DC
:104FFC003363516B536A99427ED3C91A5163282289
:10500C007A43A218517D002900D092E0117D554EB3
:10501C00C900891908688001800908603E2B75D980
:10502C001F201840454268415909091A107D8A060B
:10503C008021C0008019056809062A430A430260D2
:10504C002821794361188A8B9BB2896A206800F009
:10505C0073FBCFE0434AED00AD182B689B019B0915
:10506C002B60337DDB009B188022196812060A43E3
:10507C001A6028227A43A218517D137D002924D16D
:10508C003848DB001B185968890189095960137D60
:10509C008022DB001B18596812060A435A60282527
:1050AC007D4365192000297D03F01FF8019B002B1F
:1050BC0000D19FE02A7D236892009B181968254A2D
:1050CC001140294A0A431A6094E00129E7D1254886
:1050DC00DB001B18596889B25960137DDB001B1863
:1050EC005A68DBE7039BAD005D192A68194B1A401F
:1050FC001D4B13432B606DE7002902D1030029706F
:10510C007DE700232B7053630B0078E7117D154A64
:10511C00C9008918002B05D18022086812060243A9
:10512C000A608DE701205A08184012189206086888
:10513C00F5E7012984D1117D0A4DC9004919086888
:10514C0080B20860127D1904D20052191068014314
:10515C00116075E78F8FFF07C08000008FBFFF07BE
:10516C00808000000098004080C00000FFF78EFC9B
:10517C008022F36AD20183424CD2019BF362029BE0
:10518C001340019328237B43E3185A7D002A00D057
:10519C008DE0B149ED006D182A68920192092A60E0
:1051AC0080221B7D1206DB005B1819680A431A600B
:1051BC0028227A43A218517D137D002900D084E067
:1051CC00A548DB001B185968890189095960137DB2
:1051DC008022DB001B18596812060A435A602825E6
:1051EC007D4365192000297D02F07FFF019B002B78
:1051FC0000D15FE728237B43E3181A7D23689200D4
:10520C009B181A6895490A4030215140944A0A4328
:10521C001A6063E402991B1A1140F3620191002B8E
:10522C00B0D0019B002B08D1039BAD005D192A68FF
:10523C008C4B1A408C4B13432B6028227A43A218B8
:10524C00150038352B78012BD4D1936A1B18936237
:10525C00336B1B183363516B536A994242D3C91A8F
:10526C00516328227A43A218517D002957D1117D10
:10527C00794EC900891948688001800948603E2B25
:10528C003AD91F201840454268415909091A107D26
:10529C008A068021C0008019456809062A430A4302
:1052AC004260282179436118CA8B9BB2CDE6012A52
:1052BC0000D07DE76849ED006D182A6892B22A602B
:1052CC001B7DDB005B181A6871E7012987D16248E6
:1052DC00DB001B18596889B25960137DDB001B1861
:1052EC005A687BE7002902D103002970B9E7002333
:1052FC0053632B700B00B4E7117D574AC900891812
:10530C00002B05D180224868120602434A60C8E788
:10531C0001205A081840121892064868F5E701292E
:10532C00BFD1117D4C4DC9004919486880B2486005
:10533C00127D1904D2005219506801435160B0E734
:10534C0042050DD522684949536C20000B4053642B
:10535C00FDF7C0F92900200003F091FAFFF7C4FB18
:10536C00420406D522684249536C0B405364FFF744
:10537C00BBFB8022010092011140104203D0226835
:10538C003C49536CF1E7C20418D52068026C9A436F
:10539C00026408202268136C83431364B3239B00BC
:1053AC00E25C012A03D12000E15403F0C8FA20008A
:1053BC00FDF7C4F922683049536CD6E7020512D5C3
:1053CC0008222168086C02430A6421682B484A6C45
:1053DC0002404A6421680A6C13430B642000FDF7F9
:1053EC009FF9FFF781FB020621D5216824484A6CFE
:1053FC0002404A64B3229200A15C0029EED12168DC
:10540C00086C03430B6408232168086C03430B648A
:10541C000121A1543C22236820005B6D9B081340A2
:10542C00B4229200A35003F08AFAFFF75DFB8305C8
:10543C0009D522681349536C20000B40536403F0C8
:10544C001DFAFFF751FBC00501D4FFF74DFB226895
:10545C000D49536C89E7C04600980040BF8FFF0789
:10546C00808000008F8FFF0780C00000FFFB0000D2
:10547C00FFBF0000FFDF0000FFEF0000FFF70000A0
:10548C007FFF0000FFFD0000FFFE0000F7B50D7868
:10549C009F4AAD0045192C6803001440CA7801924C
:1054AC00032A04D81000FAF70DFE054846430122E2
:1054BC00019202E0802292001443964A14432C601D
:1054CC000F78954DBE009E1934682C403C43144314
:1054DC0034600E7B0C78002E00D08DE08F4F4E7810
:1054EC00E400E419002E30D02668360C3604266011
:1054FC000E78CC88F600F6193768A408A4003C4353
:10550C0034600C78A4001C192668760604D526682D
:10551C002E40834D354325600C78C978A400814D0D
:10552C001B1901290BD020211C682C40614008E07C
:10553C00C022D20014430022BAE78022F9E719688E
:10554C0029400A431A600198FEBD6668360C360481
:10555C006660724C0E782000F6003619CC8877689D
:10556C00A408A4003C4374600C78E400241866681A
:10557C00B601B60966600E690C783E2E24D91F2040
:10558C0077090640300046424641BF1B634EE4009B
:10559C00A419BE06802760683F0606433E4366603A
:1055AC000C78A4001C192668760404D526682E40B5
:1055BC005D4D3543256009785C4D002916D1C0211D
:1055CC001C682C408901B1E75448E4002418002ED3
:1055DC0003D1802667683606E0E70120770806408D
:1055EC00BF196668BF0637436760D9E789005B1847
:1055FC001C6880212C40E5E7CE78A4001C19022EF3
:10560C0055D127684A4E2F403E43444F2660380000
:10561C000C78E400E4192668360C360426600E7803
:10562C000C89F600F6193768A408A4003C433460D2
:10563C000C78E40024186668360C360466600E7824
:10564C004C89F60036187768A408A4003C438027E0
:10565C0074600C784878A400324EFF011C190028A5
:10566C002AD12068384206D027682F40BC466046B5
:10567C002D4F074327600C78A4001C1927687F0660
:10568C0004D527682F40264D3D432560C0250C7856
:10569C002648A4001C192768AD0107407D4015431E
:1056AC002560097889005B181968314049E726683C
:1056BC00204F3E401643A8E72068384206D02768A2
:1056CC002F40BC466046184F074327600C78A40057
:1056DC001C1927687F0604D527682F40104D3D43C1
:1056EC0025600C78CD78A4001C19012D0CD02568F0
:1056FC002E40202575401543256009780B488900FC
:10570C005B18196801401CE725683540F3E7C04673
:10571C008F89FF07808000008F8FFF070098004063
:10572C00C0800000BF8FFF0780C000008FBFFF0745
:10573C00808100008F8EFF07F7B50324D81C23400F
:10574C001C00651EAC418008001B144C0D00121986
:10575C0004000192002C0FD1002B0CD025008000EE
:10576C0009184E5DEF00BE4001353443AEB2B34272
:10577C00F7D112181460F7BD2E78013CB446674679
:10578C006E7836023E43AF783F043743EE780435EB
:10579C0036063E43019F40C70197DBE70098004067
:1057AC00F7B50C0049780600227B012900D09BE15B
:1057BC002069A569854200D90500002A20D1ABB229
:1057CC00E28861693000FFF7B7FF2378C049DB003E
:1057DC005B181A682D0492B21A602378DB005B18F0
:1057EC001A6815431D602378BA4A9B00F318196890
:1057FC00114030224A40B8490A431A600020FEBDCD
:10580C002278E7789100236A7118022F00D040E1CA
:10581C000A68984200D336E1B04B40201A40B04B96
:10582C0013430B60236A22785B1B23629300F318EB
:10583C001B6861789C461F00ABB20193634607401E
:10584C00034200D18DE000295AD1A149D20052184F
:10585C000B00516889018909516021783E2D3FD98F
:10586C002138284047427841C9006A09C918121AE0
:10587C004868920602438020000602434A6062890F
:10588C006169ABB23000FFF757FF636921695B199F
:10589C006361236A00228B4201D95A1B2B002262BE
:1058AC006278002A4CD12278894FD200D219116823
:1058BC0089018909116021783E2B31D91F201840AC
:1058CC0045426841C9005A09C919121A086892065A
:1058DC0002438020000602430A609BB222898CE0BE
:1058EC007B4BC900C918002D03D1802248681206D1
:1058FC00C3E701206A082840121892064868BCE7E2
:10590C000129BCD17248D2001218516889B2516079
:10591C0022782904D2001218506801435160AEE776
:10592C006B4AC9008918002B03D180220868120623
:10593C00D1E701205A081840121892060868CAE7E5
:10594C00012ACAD122786248D2001218116889B291
:10595C00116022781904D2001218106801431160EA
:10596C00BBE700295ED15A49D2005218116889014F
:10597C008909116021783E2D44D91F20284003004D
:10598C00584258416A09121A5148C9000918086846
:10599C00920602438020000602430A602289ABB2C1
:1059AC0030006169FFF7C8FE636922695B196361A6
:1059BC00236A934201D95F1B2B0062782762002A6D
:1059CC0050D12278424FD200D219516889018909ED
:1059DC00516021783E2B35D91F2018404542684133
:1059EC00C9005A09C919121A486892060243802044
:1059FC00000602434A609BB2628930006169FFF77E
:105A0C009BFEF0E6324BC900C918002D03D1802251
:105A1C0008681206C0E701206A082840121892068E
:105A2C000868B9E70129B9D12948D20012181168C0
:105A3C0089B2116022782904D2001218106801432F
:105A4C001160ABE7224AC9008918002B03D18022D0
:105A5C0048681206CDE701205A0818401218920621
:105A6C004868C6E7012AC6D122781948D200121814
:105A7C00516889B2516022781904D200121850680A
:105A8C0001435160B7E717480240134802430A60CC
:105A9C0058E75B1B23620868ABB229040C4DD2009B
:105AAC005219400609D5506880B250602278D20055
:105ABC0052195068014351609EE7106880B2106023
:105ACC0022780348D200121810680143116005E7D0
:105ADC0000980040BF8FFF07808000008F8FFF076A
:105AEC00808100008F8EFF07002A22D1A3692169D3
:105AFC008B4201D95A1A0B00A2612278844DD20034
:105B0C005219516889018909516022783E2B00D8BD
:105B1C00ECE01F205909034058424341C91A8B0637
:105B2C008021D20052195068090603430B4353607D
:105B3C0075E0E378022B00D08DE000291AD1237890
:105B4C00734DDB005B191A68920192091A60226985
:105B5C0023783E2A2DD91F20510902405042424140
:105B6C00891A8A068021DB005B1918680906024332
:105B7C000A431A6062782378002A5DD1644DDB00F9
:105B8C005B195A68920192095A60226923783E2A5D
:105B9C0021D91F205109024050424241891A8A06DC
:105BAC008021DB005B195868090602430A435A60DE
:105BBC0022E05749DB005B18002A03D180221968C8
:105BCC001206D5E701205108024089181A68890687
:105BDC0011431960CEE74E49DB005B18002A03D154
:105BEC00802259681206E1E7012051080240891809
:105BFC005A68890611435960E3692278002B0ED04C
:105C0C009200B218136843490B408B4201D0002B11
:105C1C0005D11168404B1940404B0B43136023785E
:105C2C003F4A9B00F61833681340C02292015A4039
:105C3C003C4B13433360E1E5012ADDD13449DB00F1
:105C4C005B185A6892B25A6023782269DB005B18A1
:105C5C0059681204AAE70120834200D0CFE5A3695A
:105C6C0022690020934201D9981A1300A0610029DF
:105C7C0019D12278264FD200D219116889018909CD
:105C8C00116021783E2B21D91F20184045426841D4
:105C9C00C9005A09C919121A0868920602438020D1
:105CAC00000602430A6061782278002900D125E7BA
:105CBC000129B4D11648D200121851681B0489B2BC
:105CCC0051602278D200121851682FE7104AC9008F
:105CDC008918002B03D1802208681206E1E7012005
:105CEC005A081840121892060868DAE70849D200D8
:105CFC005218002B03D1802351681B0616E7012094
:105D0C0059080340C918536889061943516086E73E
:105D1C0000980040404000008F8FFF07C0800000BB
:105D2C008FBFFF0780800000F7B50324D81C2340E9
:105D3C00134C800812191C00651EAC41001B0D0091
:105D4C0004000192002C0ED1002B0BD080001218F5
:105D5C00091810680500E200D5400D550134A2B2B7
:105D6C009342F7D1F7BD019F013C40CF0197370A11
:105D7C002E706F70370C360EAF70EE700435E1E795
:105D8C00009800400F4B411E02000120994217D889
:105D9C000D4902238A4203D80C4B93429B415B4230
:105DAC0007200B490A6882431A430A600A680240BA
:105DBC00934201D00A680240981A421E9041C0B228
:105DCC007047C046FF8FD003006CDC0200366E01BA
:105DDC000020024010B50400FBF712FC034801211F
:105DEC00034A02F054F8200002F0D8FD2892000873
:105DFC00DBA50008F0B585B005000C0000AFEFF393
:105E0C0010837B6072B62D4A9368FB602C4B042880
:105E1C0002D82C4B8100CB586E468AB0117C6A4656
:105E2C00D361294B29489384294B506195611162A8
:105E3C001361B121274B1032BB60B8680023890174
:105E4C00FBF7E4FCB546002C07D0E369DB0504D076
:105E5C000121214AB86802F01AF8FB68002B07D020
:105E6C00180002F0DAFD002802D00378002B00D1D4
:105E7C001A486E468AB06A46194BD0615361FB686A
:105E8C009361114B1384174B13619121002311481B
:105E9C0010328901FBF7BAFC2100B5462800FFF748
:105EAC0099FF7B68002B02D162B6BFF36F8FF86845
:105EBC00FCF7F6F8BD4605B0F0BDC046FC1100205D
:105ECC00EAA500084C9500080103000000A6000894
:105EDC00050000012892000828A60008F8A5000873
:105EEC0049A6000804000001F8B501270A4E8300FA
:105EFC009D59013084003359AB4200D8F8BD686815
:105F0C00002806D0037F3B4201D102F021FD083569
:105F1C00F1E72B689847FAE760950008012270B505
:105F2C00234B032086B01A70FFF7DEFF01F04CF90B
:105F3C000420FFF7D9FF1F4C26001F4DAC420ED397
:105F4C0000F0F2FCAE4220D300F0FEFCFAF70CFAA3
:105F5C0001211A4A137B8B43137306B070BD636A1D
:105F6C000593236A0493E3690393A369029363691A
:105F7C00019323690093E368A2686168206800F0CC
:105F8C00C5FA23685C653034D7E7B26AF36A511CF2
:105F9C0001D1591C05D011003068194303D100F010
:105FAC00A9FD3036CEE70649183000F03FFFF8E780
:105FBC00761200200091000800910008680600206D
:105FCC000F8B000870B570260125040046430102B2
:105FDC00114880220918002086B004950E350395CF
:105FEC00053565430D4B0590029001900C48F61851
:105FFC002D180C4B30000095520000F087FA04224B
:10600C00737B2C74934373730134074BE402E418D1
:10601C00EE606C6006B070BD781D0020F8050020A5
:10602C00FC110020B189000878150020F0B5002083
:10603C0087B0FFF759FF214B83F308882049214B88
:10604C000A6A00251A40C0231B0413430B62FBF79A
:10605C00FBFFFCF703F9FBF737FA1B4800F0BCFA1F
:10606C00FBF7F0F80120FFF73FFF0220FFF73CFFA2
:10607C0000F09AFC154C164B80225C61154B164EA9
:10608C000593012315490493520133002000039515
:10609C0002950195009500F039FA04220700637B04
:1060AC0020009343637302F0F6FC2800FFF78AFF8D
:1060BC00320039002000FCF7B5F8C046781D0020EE
:1060CC0000ED00E0FFFF00FF6807002068060020DD
:1060DC00FC110020DE9A0008295F0008781E0020C1
:1060EC00F0B585B004001F000392EFF3108672B672
:1060FC00C368354A002B0ED080689168884217D04F
:10610C00039B3B431AD1002E02D162B6BFF36F8FB3
:10611C00102040420AE09168897B49B20133E36068
:10612C0093682161A360002E04D0002005B0F0BD5F
:10613C002169F3E762B6BFF36F8FF6E70E23897B15
:10614C00C35649B2994200DD19000A007F3201DAC8
:10615C007F21494200258B4202DD02F02AFC05001A
:10616C001A4B22000293039B310002980093019773
:10617C0000F01EFB0028D8D0EFF3108672B6A06892
:10618C00002819D0236821699C420BD0002B09D020
:10619C009B7B5BB2994200DD19000B007F3301DA67
:1061AC007F21494202F005FC002805D031000298FD
:1061BC0000F08EFB0B20ACE7002DF7D1002EF9D1AF
:1061CC0062B6BFF36F8FF5E7FC1100207712002049
:1061DC00F8B583680500002B3CD0214A92689342A5
:1061EC003BD1C368012B03D9013BC3600020F8BD30
:1061FC00EFF3108772B60169806802F0DAFB2C6845
:10620C00AC4208D10023AB60EB609F42EED162B68A
:10621C00BFF36F8FEAE7002CF4D062682368002686
:10622C0013605A6002222000637B266093436373E1
:10623C006660A660183002F09DFC0E23AC60E3563D
:10624C0020002B61E66602F026FC3900054800F0C0
:10625C003FFBCBE716204042C9E70120FBE7C046D5
:10626C00FC1100207712002070B5EFF3108572B688
:10627C000468A0421AD0002C18D06268236800264B
:10628C0013605A6002222000637B26609343637381
:10629C006660A660183002F06DFC2000E66602F025
:1062AC00FAFB2900084800F013FB70BD8268C36834
:1062BC009B1A591E8B419B188360002DF5D162B639
:1062CC00BFF36F8FF1E7C0467712002013B50400BF
:1062DC00EFF3108172B68068002808D00138A060F6
:1062EC00002902D162B6BFF36F8F002016BD1000DB
:1062FC00184307D1002902D162B6BFF36F8F10206B
:10630C004042F3E7009201932200024800F050FA59
:10631C00ECE7C046771200200123802213B5054C10
:10632C000549064800945B42D20000F0ABF800200F
:10633C0016BDC04678950008782E0020D80600209F
:10634C00F0B5050087B0EFF3108772B62E006C6FB6
:10635C008C36002C1CD10221300002F049FB0028A5
:10636C0066D02C00843400220121200002F0E4FBD2
:10637C000028F8D10023029301225242D317009235
:10638C0001932A0039007C323C4800F06FFCDAE7BC
:10639C002368AA6F6B67944200D1AB670222336803
:1063AC00134333600423E2689A43033B1343E360D3
:1063BC006368002F47D020009847EFF310830593B4
:1063CC0072B6E36801211A008A43100908423ED1D3
:1063DC00E260E3689A071AD502229343E360284BE4
:1063EC001868002813D00021026800280FD04768D5
:1063FC00BC423AD10268002931D159681A608142F5
:10640C0000D15A60002303600830FFF72DFF0222F1
:10641C0033689343059A3360DB05DB0F002A02D106
:10642C0062B6BFF36F8F002B8DD100F0C7FA8AE7ED
:10643C003368DB069ED53060002F02D162B6BFF305
:10644C006F8F07B0F0BD62B6BFF36F8FB3E7112249
:10645C009343E36020001030FFF706FFB9E70A60B2
:10646C005A688242CED15960CCE79446002A01D0BA
:10647C0011688C46010010006246B6E777120020C6
:10648C001C120020F0B5040000206067A0672000FB
:10649C0089B07C30261D0E9DE067F06708300060E7
:1064AC0040600120002D07D0287946427041FF261C
:1064BC004042B0430230FF3026008C36306001265B
:1064CC007642F7170696079700260F480393049613
:1064DC000300029620000196009400F051F8B5429A
:1064EC000CD02968B14202D0200002F093FA6B79EB
:1064FC00002B03D00123227B13432373200000F0D5
:10650C00F9FA246709B0F0BD4D630008F0B587B007
:10651C000593030058338365C365109B07270373EA
:10652C00042300250732BA434373D2190F9BBA4395
:10653C0083738B180E0085601900C5738561C56166
:10654C0004000493FBF7B8FC049BC019B8431F1A52
:10655C000E9B3A0002930D9B310001930C9B200083
:10656C000093059BFBF748FE044B65659B68AB42AB
:10657C0000D01B6E3800236607B0F0BDFC11002064
:10658C0070B50400002086B005900E98119D049003
:10659C000D98109E03900C9802900B9801900A98FD
:1065AC0000902000FFF7B2FF2B00721C01D10133C9
:1065BC0005D02B00334305D1200000F09BFA2000BE
:1065CC0006B070BD200032002B000249183000F0DC
:1065DC002DFCF4E70F8B0008022310B50400FF33E9
:1065EC00838100F0EBFD014B9C6010BDFC11002081
:1065FC000B21084A49429368D9669866802306495C
:10660C005B05486803434B6062B6BFF36F8F9368BA
:10661C00D86E7047FC11002000ED00E00D2370B522
:10662C00C356427B002B38DBD30636D180235B422A
:10663C0013431B4C4373A3691A49E2698B4207D17C
:10664C00016042601060E06111E09A42F8D01B6872
:10665C00002BF5D00E250E2645579E57B542F4D08B
:10666C00AE42F2DD5A680360426010605860A56962
:10667C008D4201D0002D00D1E568A3685A7BD2066B
:10668C0005D1DA897F2A02D9AA69002A06D0AB4241
:10669C0002D0280000F02CFB656170BD6361FCE743
:1066AC00FC110020141200200D2270B5825605003A
:1066BC00437B002A04DA7F221340437302F0AFF9C4
:1066CC000D4E0E4AB469B368944201D0002C00D12F
:1066DC00F468AB4208D05A7BD20605D1DA897F2AFE
:1066EC0002D9A269002A05D0A34202D0200000F0F2
:1066FC00FFFA2300736170BDFC11002014120020FE
:10670C0010B5511C01D1591C03D00249183000F0AE
:10671C008DFB10BD0F8B00080D2270B58256040046
:10672C00437B002A04DA7F221340437302F077F98B
:10673C008023627B5B4213431B4D6373AB691B4924
:10674C00EA698B4207D1216062601460EC6111E050
:10675C009A42F8D01B68002BF5D00E200E2620563E
:10676C009E57B042F4D08642F2DD5A6823606260D4
:10677C0014605C60AE69AB688E4201D0002E00D113
:10678C00EE68A34208D05A7BD20605D1DA897F2A5B
:10679C0002D9B269002A05D0B34202D0300000F011
:1067AC00A7FA33006B6170BDFC110020141200209D
:1067BC0070B50C0011000A4A0A4B90681860EFF390
:1067CC00108372B69568280002F03CF9049A059B78
:1067DC002800FFF795FF2000FFF70AFF70BDC046A9
:1067EC00FC11002024120020F7B50400EFF31087F1
:1067FC0072B61F22437B1A4050425041C0B20190E6
:10680C004DB2002A3CD17F3213406373200002F05A
:10681C0006F98023627B5B4213432B4EA573637393
:10682C00B3692A498B4229D1F269216062601460F4
:10683C00F4610FE09A42F8D01B68002BF5D00E20C3
:10684C0018568542F6D0A842F4DD5A68236062607F
:10685C0014605C60B4698C4201D0002C00D1F468E7
:10686C00B3689C4202D0200000F042FA7461002F01
:10687C0002D162B6BFF36F8F0198FEBDF269DCE7FF
:10688C009B071FD5A668200002F0C9F8A5733368D2
:10689C009E4209D17368266063601C607460E6E7F1
:1068AC0072689342F6D01B68002BF3D00E229A56D6
:1068BC009542F5D0AA42F3DD5A68236062601460F9
:1068CC005C60D4E7A573D2E7FC1100201412002001
:1068DC0010B500290AD1EFF30580002807D1064B2B
:1068EC009A685B699A4202D0FFF782FE10BD62B6CD
:1068FC00BFF36F8FFAE7C046FC11002010B50028DB
:10690C000AD1EFF30580002807D1064B5A699B6822
:10691C009A4202D0FFF76CFE10BD62B6BFF36F8FC8
:10692C00FAE7C046FC110020EFF3108172B6054B5C
:10693C009A68D37B013BD373002902D162B6BFF3B3
:10694C006F8F7047FC11002070B5EFF3108672B694
:10695C00134DAB68DA7B0132DA73AC69114A94429D
:10696C0001D0002C00D1EC685A7BD20605D1DA8913
:10697C007F2A02D9A269002A05D0A34202D02000A6
:10698C0000F0B6F923006B61002E02D162B6BFF3A2
:10699C006F8FEFF3108072B6FFF7B0FF70BDC0467B
:1069AC00FC11002014120020024B034A9A61DA6198
:1069BC007047C046FC1100201412002070B5EFF394
:1069CC00108572B61C4CA168E3690A68CB1A581E74
:1069DC00834149685B420A6051601340E169A268D7
:1069EC00002B05D1154B516013600A60E2610CE07D
:1069FC000E200E2610569E57B04218D0864216DD39
:106A0C005968136051600A605A60A6690B4B9E422C
:106A1C0001D0002E00D1E668A3689E4202D030005F
:106A2C0000F066F928006661FFF7E2FD70BD8B424D
:106A3C00D8D01B68D4E7C046FC11002014120020EB
:106A4C00F8B5030007000C000B4303D1FFF7B6FFAA
:106A5C000020F8BDEFF3108672B6134D134BA868E7
:106A6C001860FFF721FEA86823003A00104918307F
:106A7C0000F0DCF90423AA680400517B30000B43BE
:106A8C005373FFF7B5FDAB689A6A002AE0D18022F8
:106A9C00DB6A12069342DBD102F092F8201AC34350
:106AAC00DB171840D5E7C046FC110020241200204B
:106ABC000F8B000870B504000D00FFF7C1FF01003B
:106ACC002000631C01D1013510D00A00CB1709201E
:106ADC000021801859410A220023F9F783FB002971
:106AEC0003D180231B06984200D3014870BDC046D9
:106AFC00FFFFFF7F70B50400EFF3108572B604261C
:106B0C00437B33420DD0183002F034F8637B200005
:106B1C00B3436373FFF782FD29000548FFF7D8FEE6
:106B2C0070BD002DFCD162B6BFF36F8FF8E7C04685
:106B3C0077120020014B98687047C046FC1100206A
:106B4C00F0B5037B85B004000393EFF3108301933E
:106B5C0072B6019B02930823427B1A4207D0019B19
:106B6C00002B02D162B6BFF36F8F05B0F0BD1900D8
:106B7C00114348B2002857DB6173A368002B02D085
:106B8C00200001F054FF20002600183001F0F2FF25
:106B9C005836A56DAE4201D0002D4DD1304F002599
:106BAC00BB689C4204D1EFF305856A1E9541EDB29A
:106BBC00BE692C4A964201D0002E00D1FE68B34229
:106BCC0002D0300000F094F820007E6101F045FA0C
:106BDC00002D02D02448FFF7FFFCBB689C4238D143
:106BEC00EFF30583002B34D1237BDB070FD5019BFF
:106BFC00002B02D162B6BFF36F8F62B6BFF36F8FFB
:106C0C000423181C02DFEFF3108372B60293029870
:106C1C00FFF7EEFC039BDB07A7D562B6BFF36F8FC4
:106C2C000423181C02DFA0E77F210A401343200035
:106C3C00637301F0F4FEA0E7280001F0F8FE2800D1
:106C4C00183001F097FF00232800EB66FFF7E6FCF5
:106C5C009FE7019B002BDDD162B6BFF36F8FD9E7A5
:106C6C00FC110020141200206807002073B5069D4B
:106C7C00079E089C00950196FFF79AFD002C03D007
:106C8C00024B9B681B69236076BDC046FC1100203B
:106C9C000121044B044AC01A044BC0104343D15485
:106CAC007047C046D807002077120020ABAAAAAACA
:106CBC00C289030000207F2A11D80A4A10680028D4
:106CCC000DD00E21084A595612680020914206DB5D
:106CDC005A7BD20603D10548181A431E984101234A
:106CEC00184070473400002028120020F8050020BE
:106CFC0070B518240C4B05001E7C0C4B7443E41827
:106D0C00200001F037FF0022094B28009A55FFF7AD
:106D1C00CFFF002807D0074B20001A680649013A1C
:106D2C00D31700F083F870BDFC110020D8070020A9
:106D3C0077120020340000209D6C000870B5EFF332
:106D4C00108572B6104A114B94681868A04207D18E
:106D5C00FFF7CEFF002D02D162B6BFF36F8F70BD6F
:106D6C0000211960127C0A4B9B5C8B42F2D02000F4
:106D7C00FFF79EFF0028EDD0637BDB0602D12000DD
:106D8C00FFF7CAFC2000E3E7FC11002024120020CE
:106D9C0077120020024B1868984200D100207047EF
:106DAC003800002070B50600FFF7F4FF002810D063
:106DBC00026943693400F517121BAB41002B08DC48
:106DCC0003D1802109068A4203D2D843C017104050
:106DDC0070BD0148FCE7C046FFFFFF7F002010B5E7
:106DEC00034B1B68834201D1FDF7CCFD10BDC0469F
:106DFC002C12002030B500280ED00B4B5B6898424B
:106E0C000AD00168002907D00A694B6904694569F1
:106E1C0012196B410A614B610368426813605A6036
:106E2C0000230360436030BD38000020F0B504003F
:106E3C0015001E0085B0531C02D1731C00D17CE0E0
:106E4C00A160EFF31083039372B6002E26DBFFF7DD
:106E5C00C5FF00210090012040197141009AD31701
:106E6C0012184B413649226163610868496812184F
:106E7C004B411E00150001230293FFF78BFF070007
:106E8C00304B9C465B680193002F1DD163462360F9
:106E9C00019B63601C6063465C6027E0284B1868AC
:106EAC00596802225242D317121A8B41521BB3411A
:106EBC001100002B04DC01D1002A01D10121002397
:106ECC00636121610023D7E73869796922696369B5
:106EDC00994202DC28D1904226D9801A99417B68CC
:106EEC0038617961636027601C607C60FFF752FF3A
:106EFC0084420FD1144B1B68002B0BD1029B002B2F
:106F0C0002D1FFF76BFF00900098FFF74BFF0021B9
:106F1C00FDF7AEFC039B002B02D162B6BFF36F8F63
:106F2C002800310005B0F0BD121A8B41226163615B
:106F3C00019B9F42AAD03F68A6E700250026EFE7F9
:106F4C00F0070020380000202C120020F0B587B08C
:106F5C00EFF3108372B601932F4B1860FFF71AFFF3
:106F6C002E4F04003A687B68029203932A4B9C468E
:106F7C001D6800280FD042690669EB179A4202DCA3
:106F8C0024D1AE4222D91900226963692800121A51
:106F9C008B4122616361029803992A00EB17121846
:106FAC004B4100243A607B60634620001C60FFF775
:106FBC00F9FE2100FDF75CFC019BA34202D162B6F5
:106FCC00BFF36F8FFFF7BAFE07B0F0BDF31704964F
:106FDC000593049A059B0298039980185941002344
:106FEC0000220E4D22616361286069602000FFF76A
:106FFC0001FF019B002B02D162B6BFF36F8F200003
:10700C00A3689847EFF3108372B6034A0193136891
:10701C009B1B1360A2E7C0462C120020F007002037
:10702C0010B5EFF3108472B6FFF7D8FE02000649D4
:10703C00C3170868496880185941002C02D162B600
:10704C00BFF36F8F10BDC046F0070020F7B50400EA
:10705C00EFF3108572B603680195002B05D0002D57
:10706C005CD162B6BFF36F8F58E00122C16A806AAF
:10707C00002312184B41002B01D1012A33D90126D0
:10708C007642F71736184F41002F01DA00260027F9
:10709C0001F09AFD01220023801859418019794191
:1070AC00002902DC3BD1002839D001F08DFD0023F2
:1070BC0001228018594180197941244B994201D100
:1070CC00033030D801F080FD012200238018594193
:1070DC0002225242D31780197941121A8B41200097
:1070EC001B49FFF7A3FE236B01332363236A002B99
:1070FC000BD0002D02D162B6BFF36F8F2000236A34
:10710C009847EFF3108372B60193A5691834A54222
:10711C0001D0002D0BD1019B002BA2D0F7BD022278
:10712C005242D317DBE7802300221B06D7E7280047
:10713C0001F0BDFC0023EB66019B002B02D162B673
:10714C00BFF36F8F280001F0A6FCE7E7FFFFFF7F7E
:10715C0059700008F8B5060014001D00EFF31087F5
:10716C0072B6511C07D1591C05D1002F02D162B641
:10717C00BFF36F8FF8BD002B0DDB14001D1E05DC5B
:10718C00002B01D1002A01D10124002501225242F9
:10719C00D317A4185D41300001F0ECFC069A079B54
:1071AC00B262F36200232200336330002B000249E9
:1071BC00FFF73CFED9E7C04659700008014B036647
:1071CC007047C046A400002010B5024800F087FBB1
:1071DC0010BDC046B7A6000810B5064C064B9C4225
:1071EC0001D3002010BD2000A268616801F03BFDB6
:1071FC001434F3E7A4000020B80000200CB470B5E0
:10720C008AB002AC05000E0020220021200001F003
:10721C003BFD0223A3700D4B25616360002E13DB35
:10722C0001D0731EED180FAA20000E996561019212
:10723C0000F00EF8002E02D0002223691A700AB05A
:10724C0070BC08BC02B018470025ECE7EB8D0008B9
:10725C00F0B5436893B003900893837815009B07AF
:10726C0000D4F8E0002301930E78002E6AD0252E6E
:10727C000DD04B1C0993019B013301930399089B7F
:10728C00F0B29847002800DADFE00999ECE74E7875
:10729C008B1C0993252EEED0002304211C00099A87
:1072AC000293079309921F2C2ED8300020381028F7
:1072BC000AD8F8F707FF1D0909270909091E09094A
:1072CC00091B0925090918003300303B092B29D962
:1072DC002A2E32D108CD600622D4002B29DB2020A7
:1072EC000793044305E001231C4302E002231C43E3
:1072FC000C43099B01321E78002ED3D109922DE04C
:10730C000823F1E71023EFE77F2C1ED83300303B26
:10731C00092BDDD8600605D50A20029E7043C318E0
:10732C000293E6E70A20079E7043C31807932023B5
:10733C00DAE75B4207932823D6E72E2E05D14023AC
:10734C001C42D1D0019813B0F0BD6C2E2DD027D893
:10735C00682E31D06A2E32D04C2E30D0029B002BAE
:10736C0003DA40239C4300230293202333431A0067
:10737C00653A022A01D9612B24D10722EB1D9343D4
:10738C0008331D00AB4F0292240753D5019A029B80
:10739C0016009C18B4424FD1079B029A9E1A82E1A8
:1073AC00742EA6D07A2EA4D0D8E780231C429BD072
:1073BC0080208000044397E780235B00F6E7A0233E
:1073CC009B0091E730006338122800D9E3E0F8F70E
:1073DC0079FE0A46E2E2E2E246E2E2E2E2E2F3DDD2
:1073EC00E2E211E2AD0004CD0CAB1A7001230CAF3C
:1073FC000293C9E780CD002F00D18F4F029963060D
:10740C0001D401214942380001F057FC0290BBE73E
:10741C0020200399089B9847002816DB013C029B0F
:10742C00A342F5D3079A019B944663441B1B01931B
:10743C000794ABE7079CF2E7019B0399FB1A985D55
:10744C00089B984701360028A4DA039B9A780423FA
:10745C001343039A937001235B42019372E7230653
:10746C003FD5A30537D50722073595432F000CCF01
:10747C0004920593102325009D43059B002B3ADABB
:10748C000499059A00244B4294410493059480235B
:10749C00DB001D43ADB20CAC0A2304980599220005
:1074AC0001F016FC041B6B0665D501232A009A43D8
:1074BC001300029AA24200DCA4E0002E00D19CE052
:1074CC001022290011400B91154200D09CE0029A29
:1074DC001D0006921EE02F0008CF0493DB170593C6
:1074EC00C8E72F0008CFE205F7D5A20501D55BB29E
:1074FC00F3E71BB2F1E7049B059A1343CBD1630668
:10750C00C9D5029B002BC6D111339C43029B25008D
:10751C001C0006932A00494B1A400B921D4277D04F
:10752C00069B0133069300230B9371E010239C43BD
:10753C00063B9C46802322001A4006921C4242D0F5
:10754C0021008133FF3319401C4239D00722EB1D37
:10755C0093431F0003CB083703000B4346D1250090
:10756C0016339D43630644D5029B002B41D1173340
:10757C009C432500029C10232A001A400B921D42AA
:10758C0056D0631C002E42D022003FE010237826F8
:10759C009C461C43CEE7782B04D110229B1B1A432C
:1075AC009446C7E725200399089B9847002800DAE2
:1075BC004BE7019B023360E6082300269C46B9E7A3
:1075CC002F0001CFC8E72F008022210008CF5200E6
:1075DC00180011401442BFD08022210092001140AB
:1075EC0098B21442B8D00699D8B2B5E706239C439A
:1075FC0025000CAC6346220052E711239D43029BED
:10760C00069387E71D00B6E71D00029A931C0693AC
:10761C002B072AD4EB0709D5079B069A02949342B1
:10762C0004DD9B1A1B190293079B0693069B10E023
:10763C0006946FE7E6A60008DFA600080604000023
:10764C0020200399089B9847002800DAFDE60A9B46
:10765C0001330A930A9A079B9342F1DC069A019B29
:10766C009B1A0A9A9B18019306920B9B002B25D010
:10767C0030200399089B9847002800DAE5E6019B27
:10768C00002E12D101330193019E029B019A9B188B
:10769C009B1BA34220DC2500002D25D13D00079B20
:1076AC00069AA4199E1A019431E002330193F0B2A8
:1076BC000399089B98470028E6DAC6E6174B1D424B
:1076CC00E2D02020AB0700D50B306D0500D52D2066
:1076DC00019B01330193EBE730200399089B0136A2
:1076EC0098470028D1DAB0E60CAB013DE85C039971
:1076FC00089B98470028CFDAA7E6019B202001338E
:10770C0001930399089B9847002800DA9DE6019A9B
:10771C00A3199B1A002BF0DCB7E5C0460604000049
:10772C007047020010B50B001179012214008C4037
:10773C0021000068046924680C4200D05340002BDF
:10774C0003D08368DB68984710BD83681B69FAE730
:10775C0010B5022901D1F9F7C9F810BDC9004018BC
:10776C00408840087047F8B50D000400FFF7F6FF9D
:10777C00F8F7FAFC1F21091A8A00A218EB0010690D
:10778C001F1D0633E719E318AEB2002808D10130EB
:10779C008840E1680143E16015613E801E80F8BDC0
:1077AC00C1000431625A3A80D200A2181880D680E7
:1077BC006652F4E70723F7B50027043ACC1D891865
:1077CC009C4399430B1BDE080460A660E760300005
:1077DC00009301912425F8F7C7FC20222D1A121AC8
:1077EC00200039009200103001F04EFA0123AD0058
:1077FC000735ED086A001A436280711BEA00A01875
:10780C004B0027804380009BA552E218019B5780B8
:10781C0019800123F600A61972882900134373807E
:10782C002000FFF7A0FFF7BDF0B585B00D001C1EC2
:10783C000290039229D000265B780193E07823789C
:10784C0040009B00C018A378C0182018019B9E42D2
:10785C0010D36279237912021A43A37903991B047A
:10786C001343E279029812061A4323000833A847FF
:10787C0005B0F0BD0378471C9B0038001F51F8F78A
:10788C00FDFC013038180136E0E716204042EFE7E6
:10789C0070B500240200012520001378002B01D1C3
:1078AC0018000AE0002813D08C4207D1702B04D0AA
:1078BC001E00403E3A2E0BD8002070BD1E00403EEC
:1078CC003A2E05D8537801320134002BE8D0002031
:1078DC00252B00D168400132DFE7002070470FB440
:1078EC0007B504A901C9019100F080FA03B008BCE6
:1078FC0004B0184770B5056908242E000023020057
:10790C0026401800254205D1D0681368984203D947
:10791C00C31A30000B6070BD126A0120D31AF9E74C
:10792C0013B501A90400FFF7E5FF002804D0019B63
:10793C00E268013B9B180193206A019BC01A013835
:10794C0016BD10B5040050182269236AD20702D55F
:10795C00013B184010BD9842FCD3C01AFAE710B591
:10796C0004000A00C168FFF7ECFF08222369E060FD
:10797C009343236110BD022270B50D008B001A4396
:10798C000368C1699B005A50040001682A00FFF784
:10799C00D8FFE3682060984203D10823226913437F
:1079AC0023612A0061682000FFF7CBFF606070BD87
:1079BC00F0B51F00C3681600C2699B00D518D25CD5
:1079CC00032385B01A40040000230291022A08D038
:1079DC0033603B600222236913420DD100230193D3
:1079EC0039E02968336089083B60F3D0FFF7B7FFB3
:1079FC00E368A3600123F2E7A369280098472B787A
:107A0C000090DA07D10F0191002AE7D002221A4028
:107A1C0003920222134221D0029B002B03D01900A7
:107A2C002000FFF7A8FF61682000009AFFF789FF8C
:107A3C00A368E1686060994206D12000009AFFF7C4
:107A4C0080FF0023A0600193A36822692360E36098
:107A5C00082313432361019805B0F0BD2000009961
:107A6C00FFF77DFFE368A360029B002B04D0236823
:107A7C00E26903999B009950029B009A9C466244D0
:107A8C003A6021682000FFF75CFF08232269206020
:107A9C001343012223612B7893432B703560A9E7A4
:107AAC0070B504000D001600FFF74BFF23688342EE
:107ABC0005D10822236925609343236170BD0223FD
:107ACC00B2001343E269AD00AB5061683200200094
:107ADC00FFF737FF6060F1E770B5036904005B07DF
:107AEC0006D5456AFFF71CFF854200D2050065628A
:107AFC0070BD70B50D0004001C22002101F0C4F80B
:107B0C000022EB68A361AB6863612B68E3616B686F
:107B1C00626223622A69002B04D0591E0B4201D1E8
:107B2C0001231A432261200001220021283000F099
:107B3C0052FF70BDF0B58BB0059300230492026A1E
:107B4C0004001E000291079309938A423BD30193D0
:107B5C00EFF3108772B6099A0397002A05D020001C
:107B6C000199FFF79DFF00230993200008A9FFF757
:107B7C00C1FE089B029A0500009393422BD3236805
:107B8C00E2699B00D618D35C0322934333702168BF
:107B9C002000029AFFF7D5FEE3682060984215D0CA
:107BAC000025039B002B02D162B6BFF36F8F0799A0
:107BBC00002906D06369002B01D0200098470023D0
:107BCC000793002DC4D130000BB0F0BD08222369FF
:107BDC0013432361E4E7002804D020000099FFF749
:107BEC00CAFEDEE7049B059A134317D000F00CFF86
:107BFC00002813D1002F11D162B6BFF36F8F200074
:107C0C00049A059B2830FEF761FB0500EFF3108307
:107C1C0072B603936B425D41EDB2C2E7236820005C
:107C2C000193009909AB07AAFFF7C2FE0500B8E75C
:107C3C0070B50400836908000D0098470200EFF34B
:107C4C00108672B60123297820000B432B706168D3
:107C5C00FFF777FE60602000FFF73EFF002E02D199
:107C6C0062B6BFF36F8F70BDF8B50400EFF31087E9
:107C7C0072B608212269A3680A4203D16168CA1A44
:107C8C008B4201D9226AD21AE169002A07D1002F4E
:107C9C0002D162B6BFF36F8F00263000F8BD9B0097
:107CAC00CE180322CB5C03211A400B42EFD0022AE0
:107CBC0002D13568AD0805D1DA0713D43000A369B9
:107CCC0098470500A1682A002000FFF73AFE29001A
:107CDC00A0602000FFF743FE002FC7D162B6BFF3B0
:107CEC006F8FC3E7022213433370A3693000A5687A
:107CFC009847290002002000FFF723FEA060002F08
:107D0C00CBD162B6BFF36F8FC7E7F8B504008369B8
:107D1C0008000D0098470600EFF3108772B6012299
:107D2C002B7893432B7023699B0705D5E268E36995
:107D3C0092009B189D421AD102222B7893432B70F0
:107D4C00A368E168994204D132002000FFF7F9FDE5
:107D5C00A06031002000FFF702FE002F02D162B6B6
:107D6C00BFF36F8F20002830FEF77EFAF8BD032298
:107D7C002E68830016401E432E60EEE710B5EFF31D
:107D8C00108472B6036982681B0703D441688B1A8E
:107D9C008A4201D9036A9B1A002C02D162B6BFF346
:107DAC006F8F5A1E9341D8B210BD704703780200F2
:107DBC0000205B070AD4136852881B035B0D120961
:107DCC009818072317309843033080087047002019
:107DDC00704710B5012100F020FF10BD10B500F068
:107DEC00F3FE0A220023F8F7FDF910BD1FB502902F
:107DFC000020039103000200010001900090F9F7AC
:107E0C009DFD05B000BD10B50120F9F711FB10BDAB
:107E1C0000207047436810B5DA710122436819607D
:107E2C0043685A71F9F7F4FA10BD70B506000C00EE
:107E3C001500081E0ED0906853681B1A99420AD878
:107E4C0013680A001818310000F015FF2000AB6809
:107E5C001B19AB6070BD1C204042FBE770B50E00D7
:107E6C00040015001900002802D1F9F7E1FA70BDE1
:107E7C00002B06D013035B0D1030C018120D00F050
:107E8C00FAFE200025606660F9F768FCEFE707B59D
:107E9C000123019201AAF9F781FC07BD07B50092F5
:107EAC0001936A460223F9F779FC07BD1FB50293CB
:107EBC00069B0192039301AA0323F9F76FFC05B00B
:107ECC0000BDF8B506000D0014001F00002C00D1F9
:107EDC00F8BD210028003A00B047241A2D18F5E708
:107EEC0010B5426804000CCA81680068FFF7E9FF0E
:107EFC00002263681A6010BD70B54B6805001A68E3
:107F0C00CB680C009A4202D10800FFF7E9FF6068C9
:107F1C00012100F082FEA3681D54002070BD70B5D5
:107F2C0004000D000A2802D10D20FFF7E5FF2900FF
:107F3C002000FFF7E1FF002070BDF0B58B6889B021
:107F4C0006930B880790DB0508000D780C005E0F7C
:107F5C001700F9F741FD0023AD0601006D0F9842A3
:107F6C0003DB2800F9F70CFC030021002268103118
:107F7C001203520D60888C18551EAA4152421140B2
:107F8C000022000904900291079806990597039422
:107F9C0001960092F9F74EFD09B0F0BD4368002040
:107FAC001B685B681961704743681B681A685268E4
:107FBC0053607047F7B5012143681B685A68117507
:107FCC001D686B682F681C685B68AE680193002C99
:107FDC0002D16B681C60F7BD21003000019AB847D4
:107FEC00241A3618F3E710B543681B681868F9F7BC
:107FFC0087FE10BD70B543680C001D686B6818696E
:10800C00F9F7F0F90F22030021002868984770BD9A
:10801C0010B500F039FE10BD10B500F02CFE10BDEF
:10802C0010B501000068F9F7E9FE10BD10B5F9F7BD
:10803C0041FFF9F75DFF10BD10B500210120F9F7E4
:10804C00DDFE10BD10B5FAF7C9F8F9F7B1FEF9F776
:10805C00BBFEFAF709F9FDF7E9FF862040427047AD
:10806C00002802D162B6BFF36F8F7047BFF34F8FFA
:10807C0030BF62B6BFF36F8F704710B50B6949699B
:10808C009847002010BD10B5FAF732F9002010BD4A
:10809C001F23012019408840704710B513000A00B7
:1080AC000121FFF7FBFE10BD10B50C00FAF79AFA90
:1080BC00002802D08460002010BD16204042FBE74F
:1080CC0070B57F240C402000FAF78CFA01000500F3
:1080DC000C312000FAF7EAFA00232B61AB68002B75
:1080EC0002D001212000984770BD70B580240C434C
:1080FC002000FAF777FA05001430FEF7B5F8AB68F4
:10810C00002B02D002212000984770BD70B5038867
:10811C000C889C4225D814889C4222D344884D88D4
:10812C00A5421ED85588A5421BD385888C88AC42A5
:10813C0017D89488AC4214D3C488CE88A64210D8E1
:10814C00D688A6420DD300890989814209D81289A3
:10815C00824206D3AB4204D80020A34200D9863811
:10816C0070BD86204042FBE770B504000D008668A8
:10817C0081683031826828003A32FFF7C7FF002847
:10818C0003D1290020003369984770BD70B50400F5
:10819C000D0083688168483182685E6C5232002E13
:1081AC0008D02800FFF7B2FF002802D129002000D8
:1081BC00B04770BD58204042FBE710B54468A46935
:1081CC00A468A04710BD10B54468A469E468A04732
:1081DC0010BD10B543689B691B69984710BD10B55D
:1081EC00FFF755FE10BD10B513000A000121FFF773
:1081FC0055FE10BD10B5FDF773FF10BD10B5FDF7A2
:10820C00E7FF10BDF0B50500066901225242D317F5
:10821C00103685B03000FFF7EDFF1821280003AAB7
:10822C00FAF734FC041E14D10127039A18213A439F
:10823C0028000392FAF740FC041E0AD100F0C4FC9B
:10824C00009001912800182103AAFAF71FFC041EC4
:10825C000CD03000FFF7D2FF200005B0F0BD182184
:10826C00280003AAFAF712FC00281BD1039B3B42FF
:10827C00EFD100F0A9FC009A019B801A99410029CA
:10828C0004DCECD1FA239B009842E8D90123039A31
:10829C0018219A4328000392FAF70EFC041ED8D139
:1082AC000B3CD6E70400D4E7F7B506690700337931
:1082BC000D00002B41D1103601225242D317300051
:1082CC00FFF798FFF023F820EC88A988013C2401E3
:1082DC001C404B1E40011B0203400F201C432B88EB
:1082EC002A89013B03401C43531E180401940400CB
:1082FC00F820400304402000019C9BB20443012B56
:10830C0010D86B885B1801335A437F2A00D97F221F
:10831C00482138001202FAF7CFFB051E08D1802342
:10832C001B041C4322000C213800FAF7C5FB050086
:10833C003000FFF763FF2800FEBD10256D42FAE701
:10834C00072300200B607047F7B506000C001500E2
:10835C0000290BD0442101AA0769FAF797FB0028E2
:10836C0007D13B79002B05D104332370002D13D199
:10837C000020FEBD019B1A0601D50323F5E79A06E2
:10838C0001D50223F1E7402219001140134201D01C
:10839C000123EAE72170E9E74021300001AAFAF74E
:1083AC0075FB0028E5D1019B2B705B045B0E6B7099
:1083BC00DEE74368DB69002901D0987B7047587B66
:1083CC00FCE703699960DA60704737B5040005690A
:1083DC0001225242D31710352800FFF70BFF18214A
:1083EC00200001AAFAF752FB002807D10222019BB8
:1083FC0018211A4320000192FAF75EFB2800FFF7C0
:10840C00FDFE37BD40689B08406C9B004068091816
:10841C005B18521A994201D10020704708685050DD
:10842C000431F7E740689B08406C9B0040680918D2
:10843C005B18521A994201D100207047505801C163
:10844C00F8E7436892085B6C92005B68C9180023DC
:10845C0052188A4201D10020704708C1F9E7002266
:10846C0010B511001520F9F78FFE1520F9F780FED5
:10847C00002216201100F9F787FE1620F9F778FE76
:10848C0010BD7047436800205B681B690B60704728
:10849C0043685B6858694240114041405961002073
:1084AC007047436800205B689961704743680020FF
:1084BC005B6899627047436800205B685A69514059
:1084CC005961704710B503699868002821D088421B
:1084DC001BD10868DC689860A14200D1D8600020EC
:1084EC000860824206D09A680A60DA689960002AAD
:1084FC0000D1D960002010E0814206D108682060CC
:10850C00D8688142EBD1DC60E9E704000068002800
:10851C00F2D1002AE7D11620404210BDF0B5012659
:10852C00302485B0029333001440019494098B409D
:10853C0034408C4040680236456803279D432C43E9
:10854C0044608468A4461C008C406643F543039544
:10855C00D5093D4065432F006546B5432F438760E1
:10856C000327520A3A406243C568B5432A43C260A6
:10857C00019A202A0CD1072914D823008B408B4058
:10858C000F215943026A8A4302994B4313430362F6
:10859C00019B02681B095C43039B1A401443046053
:1085AC0005B0F0BD0F211B0A5B435B435943426A84
:1085BC008A4302994B431A434262E9E71300F7B529
:1085CC0080221F00920217400C000197134220D00A
:1085DC009A0717D55A0765D55022D90614D580218C
:1085EC0089000A43C02519008026ED002940F600B9
:1085FC00B1424AD0A94218D08025AD00A94217D16A
:10860C00802114E01022E8E79906EBD58021C900FF
:10861C00E7E73022D903E5D5DA0603D49A06D20F60
:10862C009202DFE780229200DCE7C02149000A4376
:10863C00C0211E0089020E40056900960B420AD02B
:10864C002E693100E1408C46012167460F4202D170
:10865C00A140314329610199002906D041681E03CC
:10866C0015D50123A34049688B6100232100406884
:10867C00FFF754FF009B002B05D12B690122190039
:10868C00E14011420AD10020FEBD8021CEE75B0300
:10869C00EBD50123A34049688B62E6E7A2409343E4
:1086AC002B61F0E786204042EEE770B50B0089683D
:1086BC000500002903D05E680C68002900D170BD4C
:1086CC008B681A002A402B4202D030004B68984726
:1086DC00231E00D0236821001C00EEE7F8B505002E
:1086EC0040681F000E001400FFF718FF112F06D171
:1086FC0001236A68B3405268240502D593610020B7
:10870C00F8BD9362FBE730B5036813600579046824
:10871C00ED006419A34202D30220404230BD5C79C3
:10872C008C4201D00833F0E70020F7E74068CB0318
:10873C0000681B0D1B181F2001401E3888401B6849
:10874C000340591E8B410020137070474268CB03C5
:10875C0012681B0D9B181F2211401E3A8A40186884
:10876C0002431A600020704742681F20CB0301406F
:10877C001E38884012681B0D9B181A6882431A60B9
:10878C000020704770B50D000400FFF7DFFF2900D3
:10879C002000FFF7E9FF002070BD8022030052018A
:1087AC000800934207D080225205934207D14342DE
:1087BC00584101307047434258410330FAE7434275
:1087CC0058410230F6E7012210B5436802211B68BC
:1087DC00D869DC69C0081040144200D00843DC6939
:1087EC0004220C4200D01043D969114201D020223E
:1087FC0010438022D9695200114202D008211A621A
:10880C000843C20701D508221A62820701D501224A
:10881C001A62420701D502221A62820601D504228D
:10882C001A6210BD802210B543681B68D8691042CB
:10883C00FCD0EFF3108072B6DC69144205D100282D
:10884C00F4D162B6BFF36F8FF0E79962002800D0C5
:10885C0010BD62B6BFF36F8FFAE7082243681B683E
:10886C00D869104200D01A62DA69920603D500204A
:10887C005B6A0B70704701204042FBE7704770B594
:10888C00A525AD00435D04000220012B07D0012378
:10889C0063552068617400F053F80020605570BD7A
:1088AC0070B5040007200D000840282141436DB22B
:1088BC006618002D18DA01251431611875750870C9
:1088CC000A61CB70022B01D100230B71A525AD00E1
:1088DC00635D0220012B06D0012363552068FCF751
:1088EC00D5FD0020605570BD002555315636FF3141
:1088FC00FF3661183570E2E7F8B5072421402134C2
:10890C004C4306193700FC373B67330000255633C0
:10891C005536FF33FF3655347D67FA66FF341D70CC
:10892C00317001190068FCF73BFF2800F8BD0723E4
:10893C000B40282159434018FC30406F704770475A
:10894C00002901D18023C36400207047406C70471C
:10895C0010B543690400002B07D100230122E16804
:10896C00487802434A70584210BD98470028F4D00A
:10897C00C21783185340FF2B00DDFF23E2681370EE
:10898C00ECE7002809D00123C26800205178194275
:10899C0002D010784242504118407047EFF31083D8
:1089AC0072B6FEE710B5EFF3108372B6FFF75EFBFD
:1089BC00F9E70E2210B5825600238A4202D0FDF749
:1089CC0013FF0300180010BD030000209860D8604E
:1089DC001B605B607047002A07D08A4205D3816018
:1089EC00C260006040600020704716204042FBE7E8
:1089FC00012230B5140003688C401D00CB40A54308
:108A0C0005601800104030BDEFF30580431E9841FF
:108A1C00C0B270475820404270470020704703682E
:108A2C00426813605A60002303604360704710B5BE
:108A3C000400FFF7F4FF0222637B9343637300236C
:108A4C00A36010BD70B504000D00FDF72DFE0223D0
:108A5C00627B13436373002D1CD0A5602B689D4271
:108A6C0009D16B68256063601C606C6012E06A68F9
:108A7C009A42F6D01B68002BF3D00E220E21A25680
:108A8C0059568A42F3D09142F1DD5A6823606260F4
:108A9C0014605C6070BD10B5EFF3108472B6FDF716
:108AAC00BDFD002C02D162B6BFF36F8F10BD10B5A7
:108ABC00EFF3108472B68368002B01D0FFF7B7FF79
:108ACC00002C02D162B6BFF36F8F10BD70B50400DD
:108ADC00EFF3108572B62823427B1A420BD18368C0
:108AEC00002B01D0FFF7A3FF0422637B20009343EC
:108AFC006373FDF793FD002D02D162B6BFF36F8F48
:108B0C0070BD10B501211838FFF7E0FF10BD70B52E
:108B1C00EFF3108572B60468A0420BD0002C02D083
:108B2C002000FFF784FF002D02D162B6BFF36F8FD8
:108B3C00200070BD0024F6E7030070B5EFF310853C
:108B4C0072B604680020A3420ED084420CD0E166B9
:108B5C0022612000FFF76BFF2000183000F00AF8AC
:108B6C002000FDF75BFD0120002D02D162B6BFF3A2
:108B7C006F8F70BD70B50400EFF3108572B603688B
:108B8C00002B1AD0FEF706F906002000FEF732F98A
:108B9C00802300221B0622616361A64206D1FEF7E8
:108BAC001DF9FEF7FFF80021FBF762FE0020002DF7
:108BBC0002D162B6BFF36F8F70BD16204042F6E74C
:108BCC0010B5FEF72DFA10BD10B5FEF729FA10BD41
:108BDC004262020000231832016203638261C261A7
:108BEC00036043604363704710B50400FFF7C2FF96
:108BFC00002811D1636A002B01D020009847200077
:108C0C001830FFF784FF002806D0FFF744FFEFF37E
:108C1C00108072B6FDF772FE10BD0300EFF31082E8
:108C2C0072B6006841181960002A02D162B6BFF30F
:108C3C006F8F70470300EFF3108272B60068411A11
:108C4C001960002A02D162B6BFF36F8F7047030020
:108C5C00EFF3108272B600681960002A02D162B676
:108C6C00BFF36F8F7047030010B50C33C360036103
:108C7C00FEF7A0FD10BD002310B59A4200D110BD27
:108C8C00CC5CC4540133F8E703008218934200D142
:108C9C00704719700133F9E730B50500101E0BD081
:108CAC000024013A2B5D085D834204D1A24202D01C
:108CBC000134002BF6D1181A30BD030041188B4239
:108CCC0002D01A78002A01D1181A70470133F6E73E
:108CDC00F0B50D003721C91A8FB0C9B20D911F2103
:108CEC0004000B400C930C99E3B2082955D01029C1
:108CFC0000D164E0E9076008084369080690079111
:108D0C00A008A9070843A90808900991089E099F83
:108D1C0006980799801979410E07B4460609009602
:108D2C006646009F37430E0900970196009E019FEF
:108D3C00801979410E06B4466746060A3E430296F0
:108D4C000E0A0396029E039F801979410E04B446C5
:108D5C006746060C3E4304960E0C0596049E059F32
:108D6C008019794100260A910B960A9E0B9F801957
:108D7C0079414E07CD080521C408344361434900AD
:108D8C005B1ADBB2092B12D9012000210A3B2418F3
:108D9C004D41DBB21DE00200A5E707210B4069073E
:108DAC008C466646E008E908064334000D00303373
:108DBC0013702300501C2B43EDD10FB0F0BD0F21CD
:108DCC000B4029078C4666462009290906433400C6
:108DDC000D00092BEBD90D99CB18DBB2E7E70B692A
:108DEC004A69934202D05A1C0A61187070470000FD
:0C8DFC0001480068704700003C0800209F
:088E08008E74FF7F01000000E1
:108E100000000000A88E00081512000800000000E5
:108E2000E57100080000000000000000C88E000886
:108E300000000000A88F000800000000888F0008D4
:108E400000000000E88E000800000000488F0008C5
:108E500000000000088F000800000000688F000874
:108E600000000000288F0008912300080000000087
:108E700000000000C88F0008713F000800000000DB
:108E8000E547000800000000F5120008000000009F
:108E900025230008000000002563000800000000F2
:088EA00000000000E88F00084B
:108EA8008DA40008000000009091000854000020E4
:108EB80000000000813D00080000000000000000E4
:108EC800EEA40008BC94000880910008620000200D
:108ED800000000000000000000000000000000008A
:108EE800D49D000800000000000000005000002091
:108EF8000000000015250008000000000000000028
:108F08009AA40008DC9300085C9100085600002031
:108F18007C110020754000080000000000000000DF
:108F2800A8A40008F09300085C91000858000020ED
:108F380090110020754000080000000000000000AB
:108F4800B6A40008049400085C9100085A000020A8
:108F5800A411002075400008000000000000000077
:108F6800C4A40008189400085C9100085C00002064
:108F7800B811002075400008000000000000000043
:108F8800D2A400082C9400085C9100085E00002020
:108F9800CC1100207540000800000000000000000F
:108FA800E0A40008409400085C91000860000020DC
:108FB800E0110020754000080000000000000000DB
:108FC800C0A50008C0940008AC9100086400002007
:108FD80020000020F5430008000000000000000009
:108FE80074A400082493000800910008520000208F
:108FF800F80F0020213A00080000000000000000DF
:1090080000000000458000080000000045800008BE
:1090180000000000458000080000000045800008AE
:1090280000000000458000089C9D000849230008B6
:109038009A9D000849230008989D000849230008C4
:10904800000000001D260008000000004580000800
:10905800000000004580000800000000458000086E
:10906800000000004580000800000000458000085E
:10907800000000004580000800000000458000084E
:10908800000000004580000800000000458000083E
:10909800000000004580000800000000458000082E
:1090A8000000000045800008E88F0008912F0008A4
:1090B800E88F0008052F0008000000004580000820
:1090C80000000000458000080000000045800008FE
:1090D80000000000458000080000000045800008EE
:1090E80000000000458000080000000045800008DE
:0890F8000000000045800008A3
:109100004D830008412D0008E53500083D2E00087C
:10911000DD2C0008413100082D34000841350008DD
:1091200055830008CF830008393B0008BF8300083F
:1091300001000000020002000100800000000001A8
:1091400080000002B582000801000000010001005B
:0C915000010010000000200010002000B2
:10915C00C9850008918400089D840008AF8400082C
:10916C00B9840008C3840008C53F0008D1840008F6
:04917C0000000000EF
:10918000398700085987000875870008918700080B
:10919000D13B0008113C000800000000413C0008E1
:0C91A0004D3D000800000000F53C0008F8
:1091AC006788000831880008D38700081546000836
:0C91BC003D410008000000000000000021
:1091C800C39E000803000000AAA3000803000000D3
:1091D80081A4000803000000BE9A000803000000F4
:1091E8006A97000804000000F29D000803000000D0
:1091F800919D000803000000B098000804000000DA
:10920800EB9A000803000000EF9A00080300000032
:10921800149C000803000000DE9A00080400000007
:10922800ABA6000803000000019800080400000035
:109238003C9E000803000000CF9A000803000000CD
:10924800D0A5000803000000359E000803000000B8
:10925800289C0008030000001D9C00080300000073
:10926800109A000804000000379C00080300000062
:109278000893000808000020039C00080100000073
:10928800010006000700020006000000888F0008A1
:1092980002000000A88F000808000000A8010020B4
:1092A80000010000137E0008B97D000802000000DC
:1092B800477F0008000000000000000000000000D8
:1092C80000000000E39B0008EB9B00080000000082
:1092D8000000000000000000F39B0008F79B000856
:1092E800FB9B0008FF9B0008F89200081808002064
:1092F800991D0008300800207512002001000000A8
:1093080001800008F37F0008C17F0008B57F0008CE
:1093180000000000A97F0008000000000000000015
:109328000000000000127A0048E801000000000078
:1093380040420F00C89300089893000800001C00E2
:109348000800030003000000030003000000000001
:109358007000B000880160026002780250030000CB
:109368006C9300080068004050B7004002000000FD
:10937800889300086B840008A89300080000000088
:109388003C000000001000000B00000058002801FD
:10939800641100208410002044100020031C0800E1
:1093A800B093000801000000B89300080200000014
:1093B800030200000000000023020000000000007B
:1093C800093900089539000811840008318400081B
:1093D8004F840008FFFF0000001400500500000043
:1093E8003400000020000000FFFF000000100050C3
:1093F800040000003400000010000000FFFF00001F
:10940800000C0050030000003400000008000000B9
:10941800FFFF0000000800500200000034000000B8
:1094280004000000FFFF00000004005001000000DD
:109438003400000002000000FFFF000000000050A0
:10944800000000003400000001000000A88F0008A0
:10945800888F0008688F0008488F0008288F000848
:10946800088F000800000000000000000000000055
:1094780000000000000000000000000000000000E4
:1094880000000000000000000000000000000000D4
:1094980000000000000000000000000000000000C4
:1094A80000000000000000000000000000000000B4
:1094B800000000000010024000380140C88E00087B
:1094C8000E060000E49400080100000000000000FF
:1094D8000000000000000000EC94000840000000BC
:1094E80000400000F494000801000000FC9400080B
:1094F800020000008104000000020000A104000036
:109508000000000000000000000000000000000053
:109518000000000000000000000000000000000043
:10952800000000000100000002000000030000002D
:10953800040000000600000007000000080000000A
:109548000900000061A600086FA6000883A60008AD
:1095580092A600089EA60008108E0008108E00082B
:10956800808E0008888E0008A88E0008A88E000843
:10957800AEA6000800010000000000000010000076
:1095880000304557532043414E204644204344432E
:1095980020436F6D706F73697465204669726D77CB
:1095A800617265207374617274696E672E2E2E0065
:1095B800537461747573204C4544206465766963FF
:1095C80065206E6F74207265616479004572726FF0
:1095D8007220636F6E6669677572696E672073744F
:1095E80061747573204C45443A20256400466169CE
:1095F8006C656420746F20696E697469616C697A3E
:1096080065205046455420636F6E74726F6C3A2023
:109618002564004661696C656420746F20696E6911
:109628007469616C697A65205553422067735F7568
:1096380073623A202564004661696C656420746F22
:1096480020696E697469616C697A652043444320B6
:1096580068616E646C65723A202564004661696CC5
:10966800656420746F20696E697469616C697A65D4
:109678002067735F7573622043414E3A202564006A
:10968800455753206669726D7761726520696E6906
:109698007469616C697A6564207375636365737353
:1096A80066756C6C79004344432041434D206465E2
:1096B80076696365206E6F74207265616479004312
:1096C80044432068616E646C657220696E697469D0
:1096D800616C697A65640050464554315F4F4E00AD
:1096E8005046455431204F4E0D0A005046455431DE
:1096F8005F4F4646005046455431204F46460D0AB6
:109708000050464554325F4F4E0050464554322073
:109718004F4E0D0A0050464554325F4F46460050A2
:1097280046455432204F46460D0A0053544154557D
:10973800530050464554313A2025732C2050464555
:1097480054323A2025730D0A004552524F523A209E
:10975800556E6B6E6F776E20636F6D6D616E640D05
:109768000A006364635F68616E646C6572005046EA
:109778004554204750494F206465766963657320D6
:109788006E6F74207265616479004661696C656406
:1097980020746F20636F6E66696775726520504626
:1097A8004554312070696E3A202564004661696C21
:1097B800656420746F20636F6E66696775726520D3
:1097C80050464554322070696E3A20256400504650
:1097D800455420636F6E74726F6C20696E6974698A
:1097E800616C697A656400504645543120257300E0
:1097F800504645543220257300706665745F636F68
:109808006E74726F6C0025733A2052583A2049449E
:109818003D30782530387820444C433D2564204637
:10982800443D25640043414E2064657669636520A4
:109838006E6F74207265616479004661696C656455
:1098480020746F207365742043414E2074696D69DC
:109858006E673A202564004661696C656420746F00
:10986800206164642043414E2052582066696C741C
:1098780065723A2025640067735F757362204341FF
:109888004E20696E7465726661636520696E6974DD
:1098980069616C697A65640063616E5F72785F63A1
:1098A800616C6C6261636B0067735F7573625F63A1
:1098B800616E0047535F55534220636C6173732098
:1098C800696E697469616C697A656420737563632C
:1098D80065737366756C6C790025733A2042756CF4
:1098E8006B20494E207472616E736D697373696F72
:1098F8006E20636F6D706C6574650025733A205334
:10990800656E64696E6720256420627974657320CA
:10991800746F20686F73742028706C616365686F5A
:109928006C6465722900496E697469616C697A6949
:109938006E672063616E646C654C696768742D633B
:109948006F6D70617469626C652047535F5553424F
:1099580020636C617373004661696C656420746F81
:1099680020696E697469616C697A652043414E208B
:10997800696E746572666163653A20256400496E94
:10998800697469616C697A696E672063616E646C79
:10999800654C696768742D636F6D70617469626C7A
:1099A800652047535F55534220696E74657266613E
:1099B8006365004661696C656420746F2073657423
:1099C8002062756C6B20494E2063616C6C62616328
:1099D8006B3A2025640067735F7573625F62756C0C
:1099E8006B5F696E5F63616C6C6261636B00677368
:1099F8005F7573625F73656E645F6672616D655FE4
:109A0800746F5F686F7374007573625F67735F75F7
:109A180073620028756E7369676E656429206368D0
:109A28006172202A207573656420666F722025256F
:109A38007020617267756D656E742E204974277386
:109A4800207265636F6D6D656E64656420746F2048
:109A58006361737420697420746F20766F69642061
:109A68002A2062656361757365206974206D617968
:109A7800206361757365206D6973626568617669D5
:109A88006F7220696E206365727461696E20636FFE
:109A98006E66696775726174696F6E732E20537490
:109AA80072696E673A2225732220617267756D6547
:109AB8006E743A25640063627072696E74665F70D2
:109AC80061636B6167650073746D33325F626163F4
:109AD8006B75705F646F6D61696E006C6F67676945
:109AE8006E67006C6F67006C6F675F6D676D740001
:109AF8004D657373616765202822257322292064C8
:109B0800726F707065642062656361757365206942
:109B18007420657863656564732073697A65206C61
:109B2800696D69746174696F6E2028257529004D07
:109B38006573736167652064726F70706564206215
:109B4800656361757365206974206578636565640C
:109B5800732073697A65206C696D69746174696FC3
:109B68006E2028257529001B5B306D0025732000A9
:109B78005B2530386C755D20005B253032753A25E1
:109B88003032753A253032752E253033752C253014
:109B980033755D200025732F003C25733E2000257A
:109BA800733A2000253032782000202020007C00E5
:109BB800256300206D657373616765732064726F38
:109BC80070706564202D2D2D0D0A1B5B306D001BF8
:109BD8005B313B33316D2D2D2D20001B5B313B3329
:109BE800316D001B5B313B33336D0065727200775A
:109BF800726E00696E6600646267006C6F675F6210
:109C080061636B656E645F75617274006C6F675F2A
:109C180075617274007573625F6465766963650067
:109C28007573625F64657363726970746F720075CF
:109C380073625F7472616E736665720072302F6151
:109C4800313A2020307825303878202072312F6141
:109C5800323A2020307825303878202072322F612F
:109C6800333A20203078253038780072332F613429
:109C78003A2020307825303878207231322F6970B8
:109C88003A2020307825303878207231342F6C72A1
:109C98003A20203078253038780020787073723A6E
:109CA8002020307825303878004661756C74696EEC
:109CB8006720696E737472756374696F6E2061646E
:109CC800647265737320287231352F7063293A20C6
:109CD80030782530387800556E68616E646C65643C
:109CE800204952516E3A2025640052657365727698
:109CF800656420457863657074696F6E2028005329
:109D0800707572696F757320696E7465727275709B
:109D18007420284952512000535053454C20696EF5
:109D280020746872656164206D6F646520646F6576
:109D380073206E6F7420696E646963617465205066
:109D48005350002A2A2A2A2A2048415244204641B0
:109D5800554C54202A2A2A2A2A00415243485F4552
:109D68005843455054207769746820726561736F51
:109D78006E2025780A002A2A2A2A2A2025732025D7
:109D88006429202A2A2A2A2A006765746F707400B9
:109D9800040C02020002436C6F636B20636F6E74E5
:109DA800726F6C20646576696365206E6F742072CB
:109DB8006561647900496E76616C6964206C696ECE
:109DC80065206E756D62657220257500696E746513
:109DD80072727570742D636F6E74726F6C6C6572CD
:109DE80040343030323138303000657874695F7310
:109DF800746D333200696E76616C69642065702019
:109E08003078253032780048414C5F5043445F45F4
:109E1800505F52656365697665206661696C656443
:109E280028307825303278292C2025640075736213
:109E38005F64635F73746D333200657874656E6454
:109E48006564007374616E6461726400696E766142
:109E58006C6964206672616D652077697468202575
:109E680073202825642D626974292043414E2049B6
:109E78004420307825302A7800696E76616C6964F0
:109E88002066696C74657220776974682025732070
:109E98002825642D626974292043414E20494420B5
:109EA800307825302A782C2043414E204944206DB3
:109EB80061736B20307825302A780063616E5F63A8
:109EC8006F6D6D6F6E006661696C656420746F20DC
:109ED8007265616420726567203078253033782098
:109EE8002865727220256429006661696C656420A2
:109EF800746F2077726974652072656720307825E1
:109F080030337820286572722025642900666169DB
:109F18006C656420746F20726561642052782046F5
:109F280049464F2068656164657220286572722011
:109F3800256429006661696C656420746F20726508
:109F48006164205278204649464F2064617461203C
:109F58002865727220256429004672616D65206942
:109F68007320746F6F20626967006661696C65644D
:109F780020746F20656E61626C652043414E2074C9
:109F880072616E73636569766572202865727220E6
:109F9800256429006661696C656420746F206C65AE
:109FA80061766520696E6974206D6F646520286527
:109FB80072722025642900756E737570706F7274E3
:109FC8006564206D6F64653A2030782530387800F4
:109FD8004D657373616765206C6F7374206F6E20B5
:109FE8004649464F30004D657373616765206C6F55
:109FF8007374206F6E204649464F31006661696C64
:10A00800656420746F2072656164207478206576B9
:10A01800656E74206669666F2028657272202564F3
:10A0280029005458204649464F20656C656D656E79
:10A0380074206C6F73740041636365737320746F6D
:10A0480020726573657276656420616464726573F5
:10A0580073004D6573736167652052414D206163DC
:10A0680063657373206661696C75726500756E73DC
:10A078007570706F727465642043414E206672611A
:10A088006D6520666C616773203078253032780002
:10A0980043414E20464420666F726D6174206E6F96
:10A0A8007420737570706F7274656420696E206EA9
:10A0B8006F6E2D4644206D6F646500646174612085
:10A0C8006C656E6774682028257A7529203E206D96
:10A0D8006178206672616D652064617461206C65C9
:10A0E8006E6774682028257A752900444C43206FD0
:10A0F8006620256420666F722043414E2046442026
:10A10800666F726D6174206672616D6500444C43C0
:10A11800206F6620256420666F72206E6F6E2D4654
:10A128004420666F726D6174206672616D650066A9
:10A1380061696C656420746F207772697465205456
:10A14800782042756666657220686561646572206C
:10A158002865727220256429006661696C6564202F
:10A16800746F20777269746520547820427566662A
:10A1780065722064617461202865727220256429E3
:10A18800006661696C656420746F20777269746514
:10A19800207374642066696C74657220656C656DE3
:10A1A800656E74202865727220256429004E6F2020
:10A1B80066726565207374616E6461726420696497
:10A1C8002066696C746572206C65667400756E73C0
:10A1D8007570706F727465642043414E2066696CB7
:10A1E80074657220666C6167732030782530327828
:10A1F800004E6F206672656520657874656E6465CB
:10A20800642069642066696C746572206C65667484
:10A218000066696C746572204944202564206F7556
:10A2280074206F6620626F756E6473006661696C76
:10A23800656420746F20636C656172206578742092
:10A2480066696C74657220656C656D656E7420282E
:10A2580065727220256429006661696C65642074E2
:10A268006F20636C656172207374642066696C7416
:10A27800657220656C656D656E7420286572722044
:10A28800256429004661696C656420746F20656ED9
:10A2980074657220696E6974206D6F64650066610B
:10A2A800696C656420746F2064697361626C6520F1
:10A2B80043414E207472616E7363656976657220DE
:10A2C8002865727220256429004661696C656420DE
:10A2D800746F206578697420736C656570206D6F84
:10A2E80064650043414E207472616E7363656976DC
:10A2F8006572206E6F742072656164790043616EC7
:10A3080027742066696E642074696D696E672066BB
:10A318006F7220676976656E20706172616D0043A7
:10A32800616E27742066696E642074696D696E6752
:10A3380020666F7220676976656E2064617461704B
:10A348006861736520706172616D006661696C6532
:10A358006420746F207365742074696D696E67205A
:10A368002865727220256429006661696C6564201D
:10A37800746F207365742064617461207068617300
:10A38800652074696D696E6720286572722025647E
:10A3980029000001020304050607080C1014182000
:10A3A800304063616E5F6D63616E0043414E2070A3
:10A3B800696E6374726C2073657475702066616968
:10A3C8006C6564202825642900436F756C64206ED1
:10A3D8006F742073656C6563742063616E5F73745A
:10A3E8006D3332666420646F6D61696E20636C6FD3
:10A3F800636B00436F756C64206E6F7420747572A4
:10A408006E206F6E2043414E20636C6F636B202873
:10A41800256429004661696C65642063616C6C2061
:10A42800636C6F636B5F636F6E74726F6C5F67658D
:10A43800745F726174652870636C6B5B315D2900B1
:10A448004661696C65642063616C6C20636C6F6342
:10A458006B5F636F6E74726F6C5F6765745F726158
:10A4680074652870636C6B5B305D290063616E40B6
:10A4780034303030363830300063616E5F73746D5D
:10A4880033326664007263634034303032313030C6
:10A4980030006770696F403530303031343030000B
:10A4A8006770696F40353030303130303000677058
:10A4B800696F403530303030633030006770696F15
:10A4C800403530303030383030006770696F403593
:10A4D80030303030343030006770696F403530309C
:10A4E80030303030300072657365742D636F6E7470
:10A4F800726F6C6C6572004661696C65642063619B
:10A508006C6C20636C6F636B5F636F6E74726F6CDF
:10A518005F6765745F726174652870636C6B656EE4
:10A528005B305D2900556E61626C6520746F207325
:10A53800657420257320746F20256400636C6F6335
:10A548006B20636F6E74726F6C20646576696365E7
:10A55800206E6F7420726561647900436F756C6456
:10A56800206E6F7420656E61626C6520284C5029DE
:10A578005541525420636C6F636B00726573657448
:10A5880020636F6E74726F6C6C6572206E6F7420CE
:10A59800726561647900257320646F6573206E6F3E
:10A5A8007420737570706F72742064726976657246
:10A5B80020656E61626C650073657269616C403418
:10A5C8003030313338303000756172745F73746DB8
:10A5D80033320048616C74696E67207379737465EF
:10A5E8006D00556E6B6E6F776E206572726F7200BC
:10A5F800756E6B6E6F776E003E3E3E205A45504832
:10A60800595220464154414C204552524F52202520
:10A61800643A202573206F6E20435055202564002E
:10A628004661756C7420647572696E6720696E7412
:10A638006572727570742068616E646C696E670A01
:10A648000043757272656E74207468726561643A4D
:10A6580020257020282573290043505520657863EC
:10A66800657074696F6E00556E68616E646C6564C0
:10A6780020696E7465727275707400537461636BCF
:10A68800206F766572666C6F77004B65726E656CCD
:10A69800206F6F7073004B65726E656C2070616E11
:10A6A8006963006F7300737973776F726B71002A37
:10A6B8002A2A20426F6F74696E67205A657068791C
:10A6C80072204F53206275696C642076342E332EC5
:10A6D80030202A2A2A0A00286E756C6C29002A66FE
:08A6E8006C6F61742A00000090
:10A6F000E7780008DB7D0008F09200080000000009
:10A70000000000009380000800000000000000002E
:10A71000000000002800002000C20100000103002A
:10A720000024F400C8000000380000203800002099
:10A73000FFFFFFFFFFFFFFFFFFFFFFFFFFFFFFFF29
:10A740000000000000000000000000000000000009
:08A75000000000000000000001
:10A7580000000000000000000000000000000000F1
:10A7680000000000000000000000000000000000E1
:10A7780000000000000000000000000000000000D1
:08A788000000000000000000C9
:04A7900000000000C5
:10A7940000000000783200200020000000000000CB
:04A7A40000000000B1
:10A7A800B8000020B80000200000000001000000F0
:10A7B8001201000200000040501D6F6003040102F6
:10A7C800030109020000000100E032040309040843
:10A7D8000345575300000024034557532067735F10
:10A7E8007573622043414E2D46440000000000006E
:10A7F8000000000000000000000000220330313299
:10A808003334353637383941424344454600000031
:0FA8180000000000000000000000000000000031
:04A8280015E015E042
:040000050800207956
:00000001FF
